:100000009EC10000CDC10000CBC10000C9C10000ED
:10001000C7C10000C5C10000C3C10000C1C10000CC
:10002000BFC10000BDC10000BBC10000B9C10000DC
:10003000B7C10000B5C10000B3C10000B1C10000EC
:10004000AFC100000C949D48ABC10000A9C10000E5
:100050000C94CB48A5C10000A3C100000C94C94773
:100060009FC100000C9493470C94694799C100000C
:1000700097C1000095C1000093C1000091C100002C
:100080000C946F488DC100008BC1000089C1000035
:1000900087C1000085C1000083C1000081C100004C
:1000A0007FC100007DC100000C94414879C100006F
:1000B00077C1000075C1000073C100000C941348A3
:1000C0006FC100006DC100006BC1000069C100007C
:1000D00067C1000065C1000063C1000061C100008C
:1000E0005FC100004E414E494E495459494E46CDDC
:1000F000CCCC3D0AD7233C17B7D13877CC2B3295DF
:1001000095E6241FB14F0A000020410000C84200BC
:10011000401C4620BCBE4CCA1B0E5AAEC59D740086
:10012000407A10F35A00A0724E18090010A5D4E8C6
:100130000000E87648170000E40B54020000CA9A59
:100140003B000000E1F505000080969800000040AB
:10015000420F000000A086010000001027000000F0
:1001600000E803000000006400000000000A000036
:100170000000000100000000002C76D888DC674FEA
:100180000823DFC1DFAE59E1B1B796E5E3E453C61A
:100190003AE651997696E8E6C28426EB898C9B6212
:1001A000ED407C6FFCEFBC9C9F40F2BAA56FA5F4BC
:1001B00090055A2AF75C936B6CF9676DC11BFCE0E4
:1001C000E40D47FEF520E6B500D0ED902E03009437
:1001D0003577050080841E080000204E0A000000CC
:1001E000C80C333333330F986E12831141EF8D21D6
:1001F00014893BE65516CFFEE6DB18D1844B381B3D
:10020000F77C1D901DA4BBE424203284725E228101
:1002100000C9F124ECA1E53D2700002100240027BE
:10022000002A002D00300033000101000004010706
:10023000010A0100002200250028002B002E0031B9
:1002400000340002010000050108010B010000203C
:10025000002300260029002C002F0032000001009E
:100260000003010601090105050505070508080841
:1002700008020202020A0A08080404040401010137
:10028000010101010103030303030303030407073F
:10029000070C0C0C0C0C0C0C0C02020202060606DD
:1002A00006060606060B0B0B0B0B0B0B0B010210C5
:1002B0002020080810204010204080020102010880
:1002C0000402010102040810204080804020100830
:1002D0000402018004020180402010080402010889
:1002E00004020101020408102040800102040810E9
:1002F00020408000000A0B02090C0D0E08070304C1
:1003000001000000000000000000000000000000EC
:1003100000000000000000000000000000000012CB
:1003200011100000000000000000000000000000AC
:10033000000000000000000000001549F5561124DF
:100340001FBECFEFD1E2DEBFCDBF00E00CBF18E093
:10035000A0E0B2E0E8EEF3EC00E00BBF02C00790D3
:100360000D92A236B107D9F724E1A2E6B8E001C0A8
:100370001D92A035B207E1F711E0CEE9D1E000E02F
:1003800006C021970109802FFE010E94CE60CD3961
:10039000D10780E00807A9F70E94064B0C94E3619F
:1003A0002FCE8CBD9DBD08959C01803E910508F027
:1003B00021C5FC018827E052FE4F8F4F0C94CE6080
:1003C000C002CD02D602DF02EC02F502FA06FA06FE
:1003D000FA06FA06FA0602030F031C03FA062903BB
:1003E00032033B03480351035A0363036C03750351
:1003F000FA067E0387039003FA06FA06FA069903C3
:10040000A203AB03FA06FA06B403C103FA06FA061E
:10041000FA06CE03DB03E803FA06F503FE0307043E
:10042000FA06FA06FA06100419042204FA062F0442
:100430003C044904FA06FA06FA06560463047004FA
:10044000FA067D048A049704FA06FA06FA06A4045A
:10045000B104BE04FA06CB04D404DD04FA06FA069D
:10046000FA0601050E051B05FA06280535054205A5
:10047000FA06FA06FA064F0558056105FA06FA0665
:10048000FA06FA06FA06FA06FA066A0573057C0504
:10049000FA0685058E059705FA06FA06FA06A005FE
:1004A000AD05BA05FA06C705D405E105FA06FA0650
:1004B000FA06EE05FB050806FA0615061E062706CF
:1004C000FA06FA06FA06300639064206FA06FA066F
:1004D000FA06FA06FA06FA06FA06FA06FA06FA061C
:1004E000FA06E604EF04F804FA06FA06FA06FA0633
:1004F000FA06FA06FA06FA06FA06FA06FA06FA06FC
:10050000FA06FA06FA06FA06FA06FA06FA06FA06EB
:10051000FA06FA06FA06FA06FA06FA06FA06FA06DB
:10052000FA06FA06FA06FA06FA06FA06FA06FA06CB
:10053000FA06FA06FA06FA06FA06FA06FA06FA06BB
:10054000FA06FA06FA06FA06FA06FA06FA06FA06AB
:10055000FA064B0654066106FA066E06770684060E
:10056000FA06FA06FA0691069A06A706FA06B406ED
:10057000BD06CA06FA06FA06FA06D706E006ED0632
:1005800081E090E0A0E0B0E0809387099093880933
:10059000A0938909B0938A09089510928B0910924B
:1005A0008C0910928D0910928E09089510928F096E
:1005B000109290091092910910929209089581E089
:1005C00090E0A0E0B0E08093930990939409A09309
:1005D0009509B09396090895109297091092980979
:1005E0001092990910929A09089583E090E0A0E092
:1005F000B0E080939B0990939C09A0939D09B093D0
:100600009E09089588E790E0A0E0B0E08093B309E8
:100610009093B409A093B509B093B609089588E7FB
:1006200090E0A0E0B0E08093B7099093B809A09360
:10063000B909B093BA09089588E790E0A0E0B0E066
:100640008093BB099093BC09A093BD09B093BE09E8
:1006500008951092C3091092C4091092C50910920E
:10066000C60908951092C7091092C8091092C909C5
:100670001092CA09089581E090E0A0E0B0E0809374
:10068000CB099093CC09A093CD09B093CE090895DE
:100690001092CF091092D0091092D1091092D2096C
:1006A00008951092D3091092D4091092D50910928E
:1006B000D60908951092D7091092D8091092D90935
:1006C0001092DA0908951092DB091092DC09109259
:1006D000DD091092DE0908951092DF091092E009F9
:1006E0001092E1091092E20908951092E309109224
:1006F000E4091092E5091092E60908951092EB09B9
:100700001092EC091092ED091092EE0908951092E2
:10071000EF091092F0091092F1091092F209089570
:100720001092F3091092F4091092F5091092F6094B
:1007300008951092030A1092040A1092050A10926A
:10074000060A08951092070A1092080A1092090AE0
:1007500010920A0A089510920B0A10920C0A109235
:100760000D0A10920E0A089581E090E0A0E0B0E03A
:100770008093170A9093180AA093190AB0931A0A43
:10078000089581E090E0A0E0B0E080931B0A909390
:100790001C0AA0931D0AB0931E0A08958CE291E0F2
:1007A000A0E0B0E080932B0A90932C0AA0932D0A2E
:1007B000B0932E0A08958CE291E0A0E0B0E080931F
:1007C0002F0A9093300AA093310AB093320A089509
:1007D0008CE291E0A0E0B0E08093330A9093340A79
:1007E000A093350AB093360A089510923B0A1092EE
:1007F0003C0A10923D0A10923E0A089510923F0A58
:100800001092400A1092410A1092420A08951092E2
:10081000430A1092440A1092450A1092460A08951B
:100820001092530A1092540A1092550A1092560AC6
:1008300008951092570A1092580A1092590A10926D
:100840005A0A089581E090E0A0E0B0E080935B0A4E
:1008500090935C0AA0935D0AB0935E0A089585E0C8
:1008600090E0A0E0B0E08093630A9093640AA093C4
:10087000650AB093660A089585E090E0A0E0B0E0D4
:100880008093670A9093680AA093690AB0936A0AF2
:10089000089589E190E0A0E0B0E080936B0A909326
:1008A0006C0AA0936D0AB0936E0A089582E390E0FB
:1008B000A0E0B0E080937B0A90937C0AA0937D0A2D
:1008C000B0937E0A089582E390E0A0E0B0E08093C8
:1008D0007F0A9093800AA093810AB093820A0895B8
:1008E00082E390E0A0E0B0E08093830A9093840AD2
:1008F000A093850AB093860A089582E390E0A0E071
:10090000B0E080938B0A90938C0AA0938D0AB093E9
:100910008E0A089582E390E0A0E0B0E080938F0A11
:100920009093900AA093910AB093920A089582E35B
:1009300090E0A0E0B0E08093930A9093940AA09393
:10094000950AB093960A089580E991E0A0E0B0E09E
:100950008093A30A9093A40AA093A50AB093A60A31
:10096000089580E991E0A0E0B0E08093A70A909319
:10097000A80AA093A90AB093AA0A089580E991E071
:10098000A0E0B0E08093AB0A9093AC0AA093AD0ACC
:10099000B093AE0A08951092B30A1092B40A10925E
:1009A000B50A1092B60A08951092B70A1092B80AC2
:1009B0001092B90A1092BA0A08951092BB0A1092C6
:1009C000BC0A1092BD0A1092BE0A08951092CB0B79
:1009D0001092CC0B1092CD0B1092CE0B089510926A
:1009E000CF0B1092D00B1092D10B1092D20B089516
:1009F0001092D30B1092D40B1092D50B1092D60BF1
:100A0000089588E592E0A0E0B0E08093CB0A90934F
:100A1000CC0AA093CD0AB093CE0A089588E592E05F
:100A2000A0E0B0E08093CF0A9093D00AA093D10ABF
:100A3000B093D20A089588E592E0A0E0B0E08093F8
:100A4000D30A9093D40AA093D50AB093D60A0895F6
:100A50008EE190E0A0E0B0E08093DB0A9093DC0AA6
:100A6000A093DD0AB093DE0A08958EE190E0A0E045
:100A7000B0E08093DF0A9093E00AA093E10AB0937C
:100A8000E20A08958EE190E0A0E0B0E08093E30AEE
:100A90009093E40AA093E50AB093E60A08951092B1
:100AA000F30A1092F40A1092F50A1092F60A0895C9
:100AB0001092F70A1092F80A1092F90A1092FA0AA4
:100AC00008951092FB0A1092FC0A1092FD0A1092EF
:100AD000FE0A089510921B0B10921C0B10921D0B16
:100AE00010921E0B089510921F0B1092200B109263
:100AF000210B1092220B08951092230B1092240BBD
:100B00001092250B1092260B089510922B0B109229
:100B10002C0B10922D0B10922E0B089510922F0B70
:100B20001092300B1092310B1092320B08951092EC
:100B3000330B1092340B1092350B1092360B089534
:100B400085E090E0A0E0B0E08093430B9093440BED
:100B5000A093450BB093460B089585E090E0A0E08C
:100B6000B0E08093470B9093480BA093490BB09350
:100B70004A0B089585E090E0A0E0B0E080934B0B35
:100B800090934C0BA0934D0BB0934E0B089584EBB8
:100B900095E1A0E0B0E08093530B9093540BA093A9
:100BA000550BB093560B089584EB95E1A0E0B0E0AF
:100BB0008093570B9093580BA093590BB0935A0BFB
:100BC000089584EB95E1A0E0B0E080935B0B9093F7
:100BD0005C0BA0935D0BB0935E0B089585E090E0F5
:100BE000A0E0B0E080936B0B90936C0BA0936D0B27
:100BF000B0936E0B089585E090E0A0E0B0E08093A4
:100C00006F0B9093700BA093710BB093720B0895C0
:100C100085E090E0A0E0B0E08093730B9093740BBC
:100C2000A093750BB093760B089510927B0B1092E6
:100C30007C0B10927D0B10927E0B089510927F0B0F
:100C40001092800B1092810B1092820B08951092DB
:100C5000830B1092840B1092850B1092860B0895D3
:100C60001092930B1092940B1092950B1092960B7E
:100C700008951092970B1092980B1092990B109266
:100C80009A0B089510929B0B10929C0B10929D0B47
:100C900010929E0B08951092AB0C1092AC0C109217
:100CA000AD0C1092AE0C08958CE390E0A0E0B0E0A3
:100CB0008093AF0C9093B00CA093B10CB093B20C96
:100CC000089581E090E0A0E0B0E08093B30C9093B1
:100CD000B40CA093B50CB093B60C08951092BB0C55
:100CE0001092BC0C1092BD0C1092BE0C08958CE3B7
:100CF00090E0A0E0B0E08093BF0C9093C00CA09374
:100D0000C10CB093C20C089581E090E0A0E0B0E087
:100D10008093C30C9093C40CA093C50CB093C60CE5
:100D200008951092D30C1092D40C1092D50C1092FE
:100D3000D60C08958CE390E0A0E0B0E08093D70C4F
:100D40009093D80CA093D90CB093DA0C089581E05D
:100D500090E0A0E0B0E08093DB0C9093DC0CA093DB
:100D6000DD0CB093DE0C08951092E30C1092E40CAD
:100D70001092E50C1092E60C08958CE390E0A0E050
:100D8000B0E08093E70C9093E80CA093E90CB0934B
:100D9000EA0C089581E090E0A0E0B0E08093EB0CD5
:100DA0009093EC0CA093ED0CB093EE0C0895109280
:100DB000FB0C1092FC0C1092FD0C1092FE0C08958E
:100DC0008CE390E0A0E0B0E08093FF0C9093000DE6
:100DD000A093010DB093020D089581E090E0A0E092
:100DE000B0E08093030D9093040DA093050DB09394
:100DF000060D0895220F331F220F331FF901E95703
:100E0000F64F10821182128213820895883591055F
:100E10000CF04BC085359105CCF4803391054CF531
:100E20008D3291059CF48C319105BCF4893191058A
:100E30006CF48E30910564F48B3091053CF400978E
:100E400029F097FD08C00297049728F481E00895DF
:100E50000F970997D8F380E00895863291053CF406
:100E6000843291059CF74F970397A8F7EFCF8997A6
:100E7000FBCF843491056CF4813491053CF78A33BF
:100E800091052CF4873391050CF7C397EDCFCD97DF
:100E9000EBCF8E34910534F48B349105BCF6875436
:100EA0009109E2CF81559109DFCF863891051CF574
:100EB000833891055CF68237910584F48F3691056D
:100EC0002CF6883691053CF4853691050CF0BECFA2
:100ED0008B559109C9CF89569109C6CF8C37910599
:100EE0003CF4893791050CF0B1CF83579109BCCF01
:100EF0008D579109B9CF803D91058CF48D3C9105BA
:100F00000CF0A4CF843991053CF4813991050CF0A3
:100F10009DCF8D589109A8CF895C9109A5CF8A3DB5
:100F200091053CF4873D91050CF090CF835D9109CC
:100F30009BCF8D5D910998CF8CB58C7F8CBD8DB585
:100F40008E7F8DBD0895AF92BF92CF92DF92EF92C8
:100F5000FF920F931F93CF93DF936C017B018B0163
:100F6000040F151FEB015E01AE18BF08C017D107B3
:100F700059F06991D601ED91FC910190F081E02D3D
:100F8000C6011995892B79F7C501DF91CF911F9182
:100F90000F91FF90EF90DF90CF90BF90AF900895AA
:100FA000FC01538D448D252F30E0842F90E0821B6F
:100FB000930B541710F0CF96089501970895FC01F4
:100FC000918D828D981761F0A28DAE0FBF2FB11D4C
:100FD0005D968C91928D9F5F9F73928F90E00895A4
:100FE0008FEF9FEF0895FC01918D828D981731F05E
:100FF000828DE80FF11D858D90E008958FEF9FEFB2
:101000000895FC01918D228D892F90E0805C9F4F87
:10101000821B91098F73992708958CE09DE0F1DF81
:1010200021E0892B09F420E0822F0895FC01A48D92
:10103000A80FB92FB11DA35ABF4F2C91848D90E0FA
:1010400001968F739927848FA689B7892C93A089DD
:10105000B1898C91837080648C93938D848D981367
:1010600006C00288F389E02D80818F7D80830895FA
:10107000EF92FF920F931F93CF93DF93EC0181E0E8
:10108000888F9B8D8C8D98131AC0E889F98980818F
:1010900085FF15C09FB7F894EE89FF896083E889C2
:1010A000F98980818370806480839FBF81E090E0B4
:1010B000DF91CF911F910F91FF90EF900895F62E41
:1010C0000B8D10E00F5F1F4F0F731127E02E8C8DDB
:1010D0008E110BC00FB607FCFACFE889F989808121
:1010E00085FFF5CFCE01A2DFF2CFEB8DEC0FFD2F08
:1010F000F11DE35AFF4FF0829FB7F8940B8FEA89F6
:10110000FB8980818062D0CF682F8CE09DE0B0CFDA
:10111000CF93DF93EC01888D8823B1F0AA89BB8936
:10112000E889F9898C9185FD03C0808186FD0CC01A
:101130000FB607FCF7CF8C9185FFF2CF808185FF3A
:10114000EDCFCE0173DFEACFDF91CF91089580E03C
:1011500090E0892B21F061DF81110E94000080E086
:1011600090E0892B49F080E090E0892B29F00E94E3
:10117000000081110E94000080E090E0892B49F07E
:1011800080E090E0892B29F00E94000081110E94EC
:10119000000080E090E0892B49F080E090E0892B0E
:1011A00029F00E94000081110C94000008958150E4
:1011B000823108F05AC0E82FF0E08827ED51F74F50
:1011C0008F4F0C94CE6003090709F508FB08FF0850
:1011D00035090A09100914091A091E0922092809E2
:1011E0002C093509300936093A09809180008F773A
:1011F000809380000895809180008F7DF9CF809149
:101200008000877FF5CF84B58F7784BD089584B53E
:101210008F7DFBCF8091B0008F778093B0000895D1
:101220008091B0008F7DF9CF809190008F7780936F
:1012300090000895809190008F7DF9CF809190006B
:10124000877FF5CF8091A0008F778093A0000895CD
:101250008091A0008F7DF9CF8091A000877FF5CF8E
:10126000809120018F778093200108958091200143
:101270008F7DF9CF80912001877FF5CFCF93DF93CA
:10128000282F30E0F901ED50FD4F8491F901E3552D
:10129000FD4FD491F901E959FD4FC491CC2399F048
:1012A000811185DFEC2FF0E0EE0FFF1FE35BFD4FB8
:1012B000A591B491EC91ED2381E090E009F480E0F8
:1012C000DF91CF91089580E090E0FACF1F93CF9304
:1012D000DF93282F30E0F901ED50FD4F8491F901A3
:1012E000E355FD4FD491F901E959FD4FC491CC2349
:1012F000A1F0162F81115BDFEC2FF0E0EE0FFF1F46
:10130000ED5CFD4FA591B4918FB7F894EC9111115C
:1013100008C0D095DE23DC938FBFDF91CF911F9162
:101320000895DE2BF8CFCF93DF9390E0FC01E355D7
:10133000FD4F249189599D4FFC0184918823C9F068
:1013400090E0880F991FFC01E75EFD4FA591B491D5
:10135000FC01ED5CFD4FC591D49161110DC09FB7AB
:10136000F8948C91209582238C938881282328835C
:101370009FBFDF91CF910895623051F49FB7F894E9
:101380003C91822F809583238C93E8812E2BEFCF85
:101390008FB7F894EC912E2B2C938FBFEACF3FB7E9
:1013A000F8948091790890917A08A0917B08B09187
:1013B0007C0826B5A89B05C02F3F19F00196A11DFA
:1013C000B11D3FBFBA2FA92F982F8827BC01CD018F
:1013D000620F711D811D911D42E0660F771F881FEE
:1013E000991F4A95D1F708958F929F92AF92BF921D
:1013F000CF92DF92EF92FF926B017C01D0DF4B0125
:101400005C01C114D104E104F104B1F0C8DF681932
:1014100079098A099B09683E73408105910588F323
:1014200021E0C21AD108E108F10888EE880E83E0B5
:10143000981EA11CB11CE5CFFF90EF90DF90CF90DC
:10144000BF90AF909F908F9008952FB7F8946091C0
:1014500075087091760880917708909178082FBF71
:101460000895CF92DF92EF92FF92CF93DF93EC013A
:10147000603282E07807CCF5653B710514F064EBCF
:1014800070E0898128E830E0281B310987FD339519
:10149000220F331F220F331F6901330FEE08FF089D
:1014A0008A8128E532E0281B310987FD3395220F18
:1014B000331F220F331F032E000C440B550B2C1926
:1014C0003D094E095F09DB0177FF02C0B0E0A0E0F3
:1014D0000E94635F24EB30E040E050E00E943D5FFB
:1014E000C20ED31EE41EF51EB601E881E03370F58E
:1014F000298188E890E0821B910927FD9395880F48
:10150000991F880F991F681779077CF02A8188E551
:1015100092E0821B910927FD9395880F991F880FF0
:10152000991F681779070CF4CB010297880F991F50
:101530004FB7F8942E2F30E0F901EE0FFF1FE20FA6
:10154000F31FE755F24F928381834FBFDF91CF9115
:10155000FF90EF90DF90CF9008951F93CF93DF938C
:10156000EC01162F8881803308F04DC061E0812F97
:10157000DADE8881282F30E0F901EE0FFF1FE20F3D
:10158000F31FE755F24F1F736081607C612B60830E
:1015900019821A822CE0622F0E94AF60829FB001F4
:1015A000112430E020E0AB01420F531FFA01EE0F8F
:1015B000FF1FE40FF51FE755F24F908196FD16C00F
:1015C0002F5F3F4F2C30310571F7813009F51092B4
:1015D000800082E080938100109285001092840048
:1015E000B19A80916F00826080936F00E8818E2FA6
:1015F00090E0FC01EE0FFF1FE80FF91FE755F24FD7
:101600008081806480838881DF91CF911F910895CC
:10161000823061F4109290008093910010929500B6
:101620001092940088BB80937100E0CF833069F4FE
:101630001092A00082E08093A1001092A500109269
:10164000A40089BB80937200D1CF8111CFCF1092BB
:10165000200182E080932101109225011092240143
:101660008ABB80937300C2CFAF92BF92CF92DF92BA
:10167000EF92FF920F931F93CF93DF936B017A0149
:10168000EC01C059D74F28813CE0389F8001399F39
:10169000100D1124A090390EB12C27FF1FC0FB01A3
:1016A0001182108288818F5F888388819801280F3A
:1016B000311D87FD3A95F6012A153B051CF48881FA
:1016C0008C30BCF180819181049680349C4908F46F
:1016D00071C0F6018081918104966EC08881980165
:1016E000280F311D87FD3A952A153B05DCF68881C8
:1016F000A801480F511D87FD5A95FA01EE0FFF1FF3
:10170000E40FF51FE755F24F808186FFCBCF88812C
:10171000F801E80FF11D87FDFA95CF01EE0FFF1FCD
:10172000E80FF91FE755F24F808160E08F73CEDD3F
:10173000B9CF808191812881A801420F511D27FDD9
:101740005A959A01FA01EE0FFF1FE20FF31FE755BA
:10175000F24F21813281820F931FF70191838083A1
:1017600088819801280F311D87FD3A95F901EE0F08
:10177000FF1FE20FF31FE755F24F808186FF21C064
:101780008881080F111D87FD1A95F801EE0FFF1FC4
:10179000E00FF11FE755F24F808161E08F73DF9119
:1017A000CF911F910F91FF90EF90DF90CF90BF905E
:1017B000AF908CCD80E49CE9F701918380838FEF1B
:1017C0008883DF91CF911F910F91FF90EF90DF9071
:1017D000CF90BF90AF900895CF93CFB7F8948091FA
:1017E0006F08811123C0ECE9F2E08491E2EEF2E0AF
:1017F0009491E82FF0E0EE0FFF1FE75EFD4FA591FB
:10180000B491EC91E92319F461E085E35FDD61E0D7
:1018100085E389DD8CB580618CBD8CB580648CBD21
:1018200061E084E380DD61E083E37DDD80916F082A
:101830008F5F80936F08CFBFCF9108958CB58C6078
:101840008CBD8CB58F7D8CBD77DBC6CF0F931F937E
:10185000CF93DF938B01EA01AB014150510944332F
:10186000510508F0E9C02230310508F0E5C048E331
:10187000429FF001439FF00D1124E80FF91FE60F7E
:10188000F71F81E080836C2F232B09F4D2C061E025
:10189000802F49DD209749F460E0802F17DDCE01CD
:1018A000DF91CF911F910F910895CF3FD10511F492
:1018B00061E0BFC0F801ED50FD4FE491E150E2312D
:1018C00008F0B2C0F0E08827E759F34F8F4F0C942F
:1018D000CE607B0C820C870C910C9B0C140DA50C1C
:1018E000AD0CB50CBF0CC90CD30CE20CEC0C140DF8
:1018F000F60C000D0A0D84B5806884BDC7BDD0E02C
:10190000C0E0CDCF84B5806284BDC8BDF8CF8091E2
:101910008000806880938000D0938900C093880005
:10192000EECF80918000806280938000D0938B0006
:10193000C0938A00E4CF809180008860809380000B
:10194000D0938D00C0938C00DACF8091B000806876
:101950008093B000C093B300D2CF8091B00080627A
:101960008093B000C093B400CACF8091900080688B
:1019700080939000D0939900C0939800C0CF80913D
:101980009000806280939000D0939B00C0939A0057
:10199000B6CF80919000886080939000D0939D0096
:1019A000C0939C00ACCF8091A00080688093A00081
:1019B0008091A0008F7B8093A000D093A900C0935A
:1019C000A8009DCF8091A00080628093A000D0935A
:1019D000AB00C093AA0093CF8091A0008860809351
:1019E000A000D093AD00C093AC0089CF80912001BE
:1019F000806880932001D0932901C09328017FCF74
:101A000080912001806280932001D0932B01C093AC
:101A10002A0175CF80912001886080932001D093A6
:101A20002D01C0932C016BCF60E0C038D1050CF0C4
:101A30003FCF802F4BDC63CFC1E0D0E030CFCF93DE
:101A4000DF93D0E0C0E0CE01E1D9882319F0CE01C8
:101A50000E94D4012196C13ED105A9F7DF91CF9113
:101A600008958FB7F89480910B0D8FBF08954F9212
:101A70005F926F927F928F929F92AF92BF92CF921E
:101A8000DF92EF92FF92CF93DF93EC016C897D8917
:101A90008E899F8988889988AA88BB88CE8CDF8C9C
:101AA0000D2C000CEE08FF08603127E2720781055B
:101AB000910529F01616170618061906ACF0A701AD
:101AC0009601C501B4010E94A060DF91CF91FF9003
:101AD000EF90DF90CF90BF90AF909F908F907F90CE
:101AE0006F905F904F9008950E94115E20E030E467
:101AF0004CE157E40E94FF5F2B013C01488E598E58
:101B00006A8E7B8EC501B4010E94115EA301920111
:101B10000E94705E4B015C01C701B6010E94115E1C
:101B20009B01AC01C501B4010E94705E0E94676018
:101B3000CCCFFC0111821082138212821582148292
:101B400017821682108611861286138614861586D1
:101B500016861786108A118A128A138A108E118EA1
:101B6000128E138E158E148E178E168E10A211A241
:101B700012A213A214A215A216A217A210A611A6B1
:101B800012A613A614A615A681E090E097A786A733
:101B900080E197E2A0E0B0E0848B958BA68BB78BB9
:101BA00008958EBD00000DB407FEFDCF8EB50895DB
:101BB000DF92EF92FF920F931F93CF93DF93EC018D
:101BC000D62E122F032FF42EE52E60E088857EDBC3
:101BD0008D2D8068E6DF89878E2DE3DF8F2DE1DF95
:101BE000802FDFDF812FDDDF61E088856FDB898576
:101BF000DF91CF911F910F91FF90EF90DF900895AB
:101C00003F924F925F926F927F928F929F92AF928C
:101C1000BF92CF92DF92EF92FF920F931F93CF93D9
:101C2000DF9300D000D0CDB7DEB79E838D83362EF4
:101C300049015A012701380101DE60E0ED81FE8192
:101C4000808544DB832DADDFED81FE81818780E0DF
:101C5000A8DF80E0A6DF80E0A4DF80E0A2DF61E013
:101C6000ED81FE81808532DB60E0ED81FE81808543
:101C70002DDB832D96DFED81FE81818780E091DF72
:101C8000F82E80E08EDF082F80E08BDF182F80E0B9
:101C900088DF202F30E050E040E03F2969017A01E1
:101CA000FE2CED2CDC2CCC24C12AFE2CED2CDC2CC3
:101CB000CC24C82A61E0ED81FE81808507DB8C247D
:101CC0009D24AE24BF24482059206A207B20A301F4
:101CD00092012C253D254E255F25632D8D819E810A
:101CE00067DFED81FE81818526960FB6F894DEBF11
:101CF0000FBECDBFDF91CF911F910F91FF90EF905D
:101D0000DF90CF90BF90AF909F908F907F906F901B
:101D10005F904F903F900895CF93DF93EC0161E087
:101D2000888501DB61E08885D1DA88DD60E088851F
:101D3000CDDA80E036DF898780E033DF80E031DF95
:101D400080E02FDF80E02DDF61E08885DF91CF919B
:101D5000BDCA8F929F92AF92BF92CF92DF92EF92C5
:101D6000FF920F931F93CF93DF93EC018B015A01E6
:101D70006901D2DF85E090E0A0E0B0E00830110515
:101D8000C1F1B4F487E090E0A0E0B0E002301105CA
:101D900081F186E090E0A0E0B0E00430110549F167
:101DA00001301105A1F488E090E0A0E0B0E021C08E
:101DB00083E090E0A0E0B0E000321105D1F05CF4E7
:101DC00084E090E0A0E0B0E00031110591F080E007
:101DD00090E0DC010EC082E090E0A0E0B0E00034D2
:101DE000110539F081E090E0A0E0B0E00038110585
:101DF00071F7582F442733272227E12CF12C00E0DC
:101E00001FE06CE6CE01FCDEB50190E080E00E94B0
:101E10000F5E25ED34E045E352E40E94705E20E061
:101E200030E04AE754E40E94FF5F28EB3EE145E0E2
:101E30005EE30E94705E4B015C0126E636E646EAF0
:101E40005EE30E94FF5F20E030E040E85FE30E9435
:101E50009A5F0E946C60603180F42CEE31E548E3BB
:101E60005EE3C501B4010E94FF5F20E030E040E87E
:101E70005FE30E949A5F0E946C60862F8F71262F0D
:101E800030E050E040E0542F432F322F222722270A
:101E90003F7144275527282B60E1CE0189DE0D2CA8
:101EA000000CEE08FF08A60133272227E12CF12CB5
:101EB00001E010E06CE6CE01A3DEE12CF12C8701FD
:101EC000E39421E030E040E050E060E0CE0198DEB5
:101ED0001FE0E12EF12C00E010E023E030E040E0D4
:101EE00050E06CE6CE018CDEE12C10E8F12E01E032
:101EF00010E020E030E840E050E06CE6CE0180DE0B
:101F0000E12CF12C8701F39420E031E040E050E037
:101F100060E0CE0175DEE12C14E0F12E00E010E06F
:101F200020E034E040E050E060E0CE0169DE2FEFD9
:101F30003FEF4FE050E064E1CE013ADE2FEF3FEF9C
:101F40004FE050E065E1CE0133DE1FE0E12EF12CE1
:101F500000E010E025E030E040E050E06CE6CE012B
:101F60004FDEE12CF12C8701F39420E03FE040E0CC
:101F700050E06CE6CE0144DE64E670E080E090E084
:101F8000DF91CF911F910F91FF90EF90DF90CF9055
:101F9000BF90AF909F908F9027CACF93DF93EC01B3
:101FA000188A198A1A8A1B8A83E590E00E94D10157
:101FB00060E086E18BD983E090E00197F1F78EA590
:101FC0008295807FEEDD8FE090E00197F1F761E090
:101FD00086E1DF91CF917AC9CF92DF92EF92FF92A3
:101FE0000F931F93CF93DF938C0183E590E00E94C2
:101FF000D10160E086E16AD983E090E00197F1F7D2
:10200000F80186A597A524E0880F991F2A95E1F786
:102010008F60C7DD8FE090E00197F1F7C4E0D0E07A
:10202000C12CD12C7601FE2CED2CDC2CCC2481E0B3
:10203000B8DDC82A2197B9F761E086E147D9F801F0
:10204000C08AD18AE28AF38ADF91CF911F910F91E2
:10205000FF90EF90DF90CF9008952F923F924F9294
:102060005F926F927F928F929F92AF92BF92CF9228
:10207000DF92EF92FF920F931F93CF93DF9300D0E5
:102080001F92CDB7DEB79C838B834B015A01190198
:10209000FA82E982FA01408051806280738020E0F8
:1020A00030E0A901C301B2010E949860181674F4CF
:1020B000F6012081318142815381C301B2010E9426
:1020C0009A5FF5016083718382839383F801408076
:1020D000518062807380F401A68DB78D208931898B
:1020E000428953890E94635F6B017C01EB81FC8113
:1020F000E458FF4F8081882309F440C0C414D504FC
:10210000E604F7040CF440C0F801C082D182E282F8
:10211000F3828B819C818E5A9F4F9C838B83FC0121
:1021200080819181A281B381F10180839183A28317
:10213000B383E981FA8180819181892B41F0C401C7
:1021400096DCEB81FC8160837183828393830F90A3
:102150000F900F900F90DF91CF911F910F91FF90F3
:10216000EF90DF90CF90BF90AF909F908F907F9037
:102170006F905F904F903F902F9008954C145D04A6
:102180006E047F040CF0C0CFF50140805180628066
:10219000738020E030E04AEF56E4C301B2010E94B0
:1021A0000B5E87FFB1CF20E030E040E85FE3C30182
:1021B000B2010E949B5FF5016083718382839383E8
:1021C000A3CFCF93DF93EC0183B183B1E0E0F1E0E3
:1021D00080818081CE018E529E4FFEDE83B183B11D
:1021E00080B180B1CE018E5F9D4FF6DE83B183B1A9
:1021F00080B180B1CE018E5C9D4FDF91CF91ECCE4E
:10220000889A0895889808958E9A08958E980895CA
:10221000EBE0F1E08081886080830895EBE0F1E0FD
:102220008081877F80830895149A08951498089573
:1022300060E0FC01878D4AC860E0FC01818D46C8E2
:1022400061E0FC01878D42C861E0FC01818D3EC8E0
:10225000CF93DF93EC01FC01EB57FF4F10823797D0
:1022600081E0808360E0898D31D88BA19CA1892B8E
:1022700029F060E08F8DDF91CF9128C8DF91CF9159
:102280000895CF93DF93EC018FA10E943E092AA508
:102290002817190621F48BA5DF91CF91089580E0CE
:1022A000FBCFCF93DF93EC018DA10E943E092AA5BD
:1022B0002817190621F48BA5DF91CF91089580E0AE
:1022C000FBCFCF93DF93EC018B8DFE01EF5BFF4FD4
:1022D000908161E0911101C060E00E94660989A1CE
:1022E000FE01EE5BFF4F9081992331F0CD5BDF4F14
:1022F000988161E0911101C060E0DF91CF910C9471
:102300006609CF93DF93EC018B8DFE01EF5BFF4FEE
:10231000908160E0911101C061E00E94660989A18D
:10232000FE01EE5BFF4F9081992331F0CD5BDF4FD3
:10233000988160E0911101C061E0DF91CF910C9430
:102340006609CF93DF93EC0161E08D8D0E946609F1
:10235000FE01EE5BFF4F8081882321F061E08BA1BD
:102360000E946609CD57DF4F1882DF91CF91089503
:10237000CF93DF93EC01FC01E45AFC4F1082EE583E
:10238000F1098081811103C0CE014096DADFFE01A0
:10239000E153FD4F8081811104C0CE018A559F4FCA
:1023A000D0DFFE01E053FD4F8081811104C0CE01DA
:1023B000845C9E4FC6DF64E670E080E090E0DF91D1
:1023C000CF9112C8CF93DF93EC0160E08D8D0E9416
:1023D0006609FE01EE5BFF4F8081882321F060E0FB
:1023E0008BA10E946609CD57DF4F81E08883DF9182
:1023F000CF9108958F929F92AF92BF92CF92DF922A
:10240000EF92FF920F931F93CF93FC01E25BFF4F7C
:102410004083518362837383349640835183628304
:10242000738334960083118322833383DC01A65A9D
:10243000BF4FEC925297CC91CC2351F018974C910E
:10244000411152C037FF56C010821182128213828E
:10245000DC01A75BBF4F4D915D916D917C9113970E
:10246000141615061606170634F514963C913323F8
:1024700011F1C080D180E280F38046015701F7FE60
:1024800007C08824992454018C189D08AE08BF0801
:10249000481559056A057B0574F4F7FE07C0709569
:1024A0006095509541955F4F6F4F7F4F40835183AB
:1024B00062837383C32FFC01E959FF4F108211829D
:1024C0001282138285589F4F31E0FC0130838C2F9C
:1024D000CF911F910F91FF90EF90DF90CF90BF9021
:1024E000AF909F908F900895101611061206130654
:1024F0000CF4AACFC0E0ACCF0F931F93CF93DF9320
:10250000EC01062F89A581110DC0CE01CADE182F5E
:10251000CE01B7DE0111182F812FDF91CF911F91CE
:102520000F910895CE01ADDE182FCE01BADEF2CFA5
:10253000CF93DF93EC01FC01E958FF4F808191813B
:10254000A281B3810196A11DB11D80839183A283D5
:10255000B3833E9681E08083AE014E5A5F4FFA010D
:1025600080819181A281B3819E0124583F4FF9015E
:102570002081222309F440C00196A11DB11DFA015A
:1025800080839183A283B383FE01E857FF4F2081AC
:102590003181C901959587958C0F9D1F32970190C8
:1025A000F081E02D20FF08C0DC012D913C91E20F6D
:1025B000F31F0190F081E02D19958BA19CA1892B2F
:1025C000F9F0FE01E457FF4F20813181C901959553
:1025D00087958C0F9D1FC657DF4FE881F98120FF3B
:1025E00008C0DC012D913C91E20FF31F0190F081B6
:1025F000E02DDF91CF9119940197A109B109BFCFC7
:10260000DF91CF9108958F929F92AF92BF92CF9218
:10261000DF92EF92FF920F931F93CF93DF93EC0122
:10262000FC01E959FF4F60817181828193810E9491
:102630000F5E6B017C01FE01EC5BFF4F60817181DD
:10264000828193810E94115E9B01AC0160E074E283
:1026500084E799E40E94FF5F4B015C01FE01ED58A5
:10266000FF4F60817181828193810E940F5E9B0187
:10267000AC01C501B4010E94FF5F4B015C018E01FA
:1026800005591F4F20E030E040E05FE30E94705E9C
:10269000A70196010E949B5F0E946C60F801608315
:1026A000718382839383C159DF4FA5019401C701D0
:1026B000B6010E949B5F0E946C60688379838A8365
:1026C0009B83DF91CF911F910F91FF90EF90DF904F
:1026D000CF90BF90AF909F908F9008950F931F93CE
:1026E000CF93DF93FC01EB57FF4F20812223B9F0FA
:1026F0007E970081118122813381389640815181FA
:1027000062817381041715072607370710F1EC0162
:102710009FDDCE01DF91CF911F910F9174CFFC010E
:10272000E558FF4F20812223A1F074970081118189
:1027300022813381349640815181628173810417F3
:1027400015072607370728F0DF91CF911F910F91CA
:10275000EFCEDF91CF911F910F910895FC01E558C5
:10276000FF4F2081222361F0749780819181A281A3
:10277000B3810196A11DB11D80839183A283B38390
:1027800008950F931F93FC01E65AFF4F20812111FA
:1027900012C03897008111812281338134964081A3
:1027A00051816281738104171507260737074CF49E
:1027B0001F910F91A6CDFC01E05CFF4F20812111FC
:1027C000F7CF1F910F917DCDCF92DF92EF92FF92C5
:1027D0000F931F93CF93DF93EC017B016A01890173
:1027E0009A01AB01B80188819981B3DA8C8188356F
:1027F00071F49601A701B8018A819B81DF91CF9185
:102800001F910F91FF90EF90DF90CF90A2CADF91C0
:10281000CF911F910F91FF90EF90DF90CF9008958F
:10282000CF93DF93EC018C818835A9F588E093E1A3
:102830009983888388E393E19B838A8384E291E18F
:10284000FE01EA57FF4F91838083329611821082F6
:1028500080E291E1329691838083329611821082D8
:102860008CE191E1329691838083329611821082BD
:1028700088E191E1329691838083329611821082B1
:102880008881998149DA8C81883589F48A819B8194
:10289000DF91CF9141CA893529F488E193E1998389
:1028A0008883CCCF8A3551F688E293E1F8CFDF9167
:1028B000CF910895CF93DF93FC01DC0116968AE057
:1028C000ED0119928A95E9F781E0808B818B138A5B
:1028D000128A148A158A168A178A108E8CE291E061
:1028E000A0E0B0E084A795A7A6A7B7A742E350E071
:1028F00060E070E040AB51AB62AB73AB44AB55AB47
:1029000066AB77AB80AF91AFA2AFB3AF88E790E093
:10291000A0E0B0E084AF95AFA6AFB7AFDF01A05C99
:10292000BF4F1C9211961C9211961C9211961C92EC
:10293000119644E650E060E070E04D935D936D9336
:102940007C93139714961C9211961D921D921D92C2
:102950001C92139714961C9211961D921D921D9213
:102960001C92139714961D921D921D921C92139700
:1029700014961D921D921D921C92139714961C92F0
:1029800011961D921D921D921C92139714961D92E2
:102990001D921D921C92139714961D921D921D92CA
:1029A0001C92139714961D921D921D921C921397C0
:1029B00014961D921D921D921C92139714961D92AF
:1029C0001D921D921C92139714961D921D921D929A
:1029D0001C92139714961D921D921D921C92139790
:1029E00014961C9211961C9211961C9211961C9290
:1029F00011961C9211961C9211961C9211961C9283
:102A000011961C9211961C9211961C92128E118E88
:102A1000148E138E168E158E10A2178E12A211A26E
:102A200014A213A216A215A210A617A2119684E250
:102A300091E111969C938E93129611961C921E9280
:102A4000129680E291E111969C938E9312961196C4
:102A50001C921E9212968CE191E111969C938E939A
:102A6000129611961C921E92129688E191E18D9316
:102A70009C93EC56FF4F11821082DF91CF91089505
:102A800008958FEF9FEF089508950895089508958C
:102A9000089508950895089508950895089508954E
:102AA000089508950895089508950895089508953E
:102AB000089580916D0890916E08892B41F481E012
:102AC00090E00E94925890936E0880936D088091D8
:102AD0006D0890916E0808950F931F93CF93DF9325
:102AE0008B01E7DFF801C2A1D3A1868D978D8530D8
:102AF000910529F14CF40497B1F090E080E0DF916A
:102B0000CF911F910F9108958630910511F10B9788
:102B1000A1F76BE070E083E49EE00E94AD0ABE0185
:102B200083E49EE009C064E070E08AE39EE00E94D6
:102B3000AD0ABE018AE39EE00E94310ADECF65E065
:102B400070E08DE39EE00E94AD0ABE018DE39EE041
:102B5000F3CF66E070E080E49EE00E94AD0ABE0123
:102B600080E49EE0E9CF8091690890916A08892B02
:102B700091F480E790E00E949258FC0131969C010C
:102B80002B5C3F4F119217AAE217F307D9F79093E6
:102B90006A08809369088091690890916A0808958D
:102BA0004F925F926F927F92AF92BF92CF92DF92DD
:102BB000EF92FF920F931F93CF93DF93EB01D3DF3D
:102BC0008C01CAA8DBA84EA45FA468A879A8AEA00F
:102BD000BFA0EE8CFF8C4AA15BA19601B7010E94B9
:102BE000260CC301B2010E94F4099601A501B701A8
:102BF000C8010E94260C90E080E0DF91CF911F91E8
:102C00000F91FF90EF90DF90CF90BF90AF907F90AB
:102C10006F905F904F900895CF93DF93EB01A3DF08
:102C20006AA98E8D0E94930990E080E0DF91CF9198
:102C30000895CF93DF93EB0196DF2AA93BA94AA120
:102C40005BA16E8D7F8D0E94260C90E080E0DF916D
:102C5000CF9108958091620890916308892BE1F5E6
:102C600085E390E00E949258FC0181E090E0A0E0B2
:102C7000B0E080839183A283B38384839583A6830A
:102C8000B78380879187A287B387158614861686B7
:102C90001786108A118A128A138A148A158A168A4C
:102CA000178A108E118E138E128E12A213A214A2E6
:102CB00015A217A216A210A611A612A613A614A654
:102CC00015A616A617A610AA11AA12AA13AA14AA24
:102CD000F0936308E0936208809162089091630822
:102CE0000895CF93DF93B6DFEC0185E40E943E099F
:102CF00021E0892B09F420E02C8FACDFEC0184E487
:102D00000E943E0921E0892B09F420E02D8FA2DFEB
:102D1000EC0183E40E943E0921E0892B09F420E0C4
:102D20002E8F98DFEC0182E40E943E0921E0892B7E
:102D300009F420E02F8F8EDFEC0181E40E943E0930
:102D400021E0892B09F420E028A384DFEC0180E452
:102D50000E943E0921E0892B09F420E029A3DF919C
:102D6000CF91089577DFBDCF75DFFC0114AA90E005
:102D700080E00895FC0101900020E9F73197AF0150
:102D8000481B590BBC018CE09DE00C94A3078F926B
:102D90009F92AF92BF920F931F93CF93DF93CDB7C4
:102DA000DEB7A1970FB6F894DEBF0FBECDBF19A254
:102DB000423008F44AE08E010F5D1F4F842E912CA3
:102DC000B12CA12CA50194010E94695FE62FB901E5
:102DD000CA01EA30ECF4E05DD801EE938D01232BBB
:102DE000242B252B79F790E080E0109711F0CD018E
:102DF000C1DFA1960FB6F894DEBF0FBECDBFDF9145
:102E0000CF911F910F91BF90AF909F908F90089599
:102E1000E95CE2CFCF92DF92EF92FF92CF93DF9304
:102E200097FF18C06B017C018DE20E948408EC01C1
:102E300066277727CB016C197D098E099F094AE027
:102E4000A6DF8C0F9D1FDF91CF91FF90EF90DF9059
:102E5000CF9008954AE0DF91CF91FF90EF90DF90FF
:102E6000CF9095CFBC01990F880B990BD3CF82CF10
:102E7000882319F08AEB97E0FACF83EB97E0FCCF39
:102E80002F923F924F925F926F927F928F929F927A
:102E9000AF92BF92CF92DF92EF92FF920F931F9368
:102EA000CF93DF93CDB7DEB762970FB6F894DEBF4E
:102EB0000FBECDBF1C018C010E5A1F4F1E870D8700
:102EC000D8014D915D916D917C917C01B6E5EB0E41
:102ED000F11CF70180819181A281B3816101FAE542
:102EE000CF0ED11CF6012081065D1F4F5801B3960D
:102EF0004F012223B9F19101205C3F4FF90120815C
:102F0000F801208321E0F40120834115510561057A
:102F1000710559F4F10100A911A922A933A9ED58AD
:102F2000FF4F00831183228333838101025B1F4F94
:102F3000F8014080518062807380910125583F4F95
:102F40005901481659066A067B06B4F54817590711
:102F50006A077B07DCF1D6018C91811137C0D5015E
:102F60001C923AC121E0481759076A077B070CF009
:102F700020E0F50120832A013B0177FF07C04424AC
:102F800055243201441A550A660A770A8C019D01BC
:102F9000B7FF07C0002711279801081B190B2A0B40
:102FA0003B0BBB24B39440165106620673060CF427
:102FB000B12CF401B082A9CF84159505A605B705FB
:102FC00054F684179507A607B7072CF6F5018081FC
:102FD000882329F2D6018C9181110DC0F6018081E0
:102FE0008111BDCFD4016C9181E06827C10184DAE1
:102FF0008111B5CF05C060E0C1017EDA8111EECF4D
:10300000D101D8962D913D914D915C91DB9729830B
:103010003A834B835C839C962D913D914D915C91BD
:103020009F972D833E834F835887D0962D913D9156
:103030004D915C91D39729873A874B875C87F7013D
:1030400080819181A281B381ED85FE85C080D18090
:10305000E280F380F8014081518162817381F10146
:10306000E158FF4F1082319610823101F1E86F0E66
:10307000711CF301108291012E573F4FF90110820C
:10308000329610824C015D01841A950AA60AB70A8D
:10309000B7FE08C0B094A09490948094811C911CB9
:1030A000A11CB11C481759076A077B072CF0C81AE6
:1030B000D90AEA0AFB0A04C0C41AD50AE60AF70AC2
:1030C000D501C401B595A795979587958D879E875E
:1030D000AF87B88B81010C571F4F8C149D04AE0431
:1030E000BF0408F09EC0D101D4960D90BC91A02DD4
:1030F000BA8BA98B81E0F9018083D8018C93F1010F
:103100008489882309F45CC00E94250AD101529663
:103110000D911C91012E000C220B330B601B710BC7
:10312000820B930B693E73408105910508F448C0FA
:103130000E94250AF101738B628B88E993E097DE88
:103140008CE993E094DE60E070E0CB0163DE82EA1C
:1031500093E08DDEC701B6015DDE88EA93E087DE8D
:10316000C501B40157DE8EEA93E081DE4AE06D8549
:103170007E858F8598890BDE85EB93E078DE69810B
:103180007A818B819C8146DE8BEB93E070DE6985D2
:103190007A858B859C853EDE81EC93E068DE6D81CF
:1031A0007E818F81988536DE87EC93E060DE82E554
:1031B00096E05DDE89899A8955DE8EE298E057DED9
:1031C000F101ED58FF4F09891A89C801B0E0A0E06C
:1031D00080839183A283B38360E0C1018DD988236A
:1031E00039F0F101EE5AFF4F1082118212821382E0
:1031F00062960FB6F894DEBF0FBECDBFDF91CF91C0
:103200001F910F91FF90EF90DF90CF90BF90AF9004
:103210009F908F907F906F905F904F903F902F90F6
:1032200008952D853E854F8558892C153D054E0501
:103230005F0508F450C089819A81AB81BC818C15EF
:103240009D05AE05BF0544F4AD81BE811196BA8BD4
:10325000A98B81E0F30150CFC701B6010E94115E36
:103260002B013C0169817A818B819C810E94115ED6
:103270009B01AC01C301B2010E94FF5F2B013C0125
:103280006D817E818F81988529853A854B855C8506
:10329000621B730B840B950B0E94115E9B01AC01AA
:1032A000C301B2010E94705E2B013C0169857A85E1
:1032B0008B859C850E94115E9B01AC01C301B2010C
:1032C0000E949B5F0E9467607A8B698B81E0F101AD
:1032D000E158FF4F11CFD501C40129813A814B81BB
:1032E0005C81821B930BA40BB50BC816D906EA06AA
:1032F000FB065CF44D815E814E5F5F4F5A8B498BBC
:1033000081E0F101EF57FF4FF7CEC501B4016C1911
:103310007D098E099F090E94115E2B013C01698184
:103320007A818B819C810E94115E9B01AC01C3015B
:10333000B2010E94FF5F2B013C016D817E818F8174
:10334000988529853A854B855C85621B730B840BB8
:10335000950B0E94115E9B01AC01C301B2010E945A
:10336000705E2B013C0169857A858B859C850E9466
:10337000115E9B01AC01C301B2010E949B5F0E94E0
:1033800067607A8B698B81E0F101E058FF4FB4CE22
:10339000CF93DF93EC018DEC93E069DD6AA17BA113
:1033A0008CA19DA137DD8EE298E0DF91CF915FCDBA
:1033B0000F931F93CF93DF938C01EB018AE793E088
:1033C00056DD82E596E053DDF80184810E94840891
:1033D000CE0148DD3FDCDF91CF911F910F91D8CF17
:1033E000EF92FF920F931F93CF93DF93182F092F24
:1033F0007B016115710569F50E943E0931E020E00D
:10340000019709F030E0C32FD22F82E0E816F104D3
:1034100008F045C080ED93E02ADD82E596E027DDE7
:1034200084ED93E024DD812F902F1CDD82E596E072
:103430001EDD8FE598E01BDDCE0114DD0BDCA8DF7F
:1034400090E080E0DF91CF911F910F91FF90EF907E
:103450000895D0E0C0E061307105B9F6812F1633D0
:1034600010F08AEC810F20917B00982F9870277FB5
:10347000922B90937B008770806480937C00809176
:103480007A00806480937A0080917A0086FDFCCF78
:1034900080917800C0917900DC2FC82FB6CF81E0F1
:1034A00090E0D0CF0F931F93CF93DF93FC01208147
:1034B000318121153105C1F1EC01822F0E943E09B5
:1034C00021E0892B09F420E02B876A85261701F17A
:1034D0001E821F82188619860E811F8128853985D4
:1034E0008A819B81AC81BD81081719072A073B0798
:1034F000DCF081E0682788810E94660934DB70E097
:1035000060E088819981DF91CF911F910F9168CF01
:103510008E819F81A885B9850196A11DB11D8E83DD
:103520009F83A887B987D8CFDF91CF911F910F9143
:103530000895CF93DF93EB0116DB6AA97BA98E8DEB
:103540009F8D4EDF90E080E0DF91CF910895CF9284
:10355000DF92EF92FF92CF93DF93EB01CB010E94BA
:103560000607882351F1FE01EE0FFF1FEE0FFF1F2C
:10357000E957F64FC080D180E280F38086ED93E07A
:1035800076DC82E596E073DC84ED93E070DCCE01BE
:1035900069DC82E596E06BDC8FE598E068DCC701CA
:1035A000B60138DC57DBF4DE90E080E0DF91CF91AC
:1035B000FF90EF90DF90CF9008958AED93E057DC75
:1035C000F3CF0F931F93CF93DF938C01D0E0C0E034
:1035D000CE010E940607882319F0BE01C801B7DF9B
:1035E0002196C13ED105A1F7DF91CF911F910F9197
:1035F00008958CEF93E03BDC8AE292E038DC8AE0CD
:1036000092E035DC81E094E032DC24DBC1DE90E046
:1036100080E00895CF93DF93EC018BE094E027DC0A
:103620008FE094E024DC8C8D23DC83E194E01FDCCC
:103630008D8D1EDC87E194E01ADC8E8D19DC8BE128
:1036400094E015DC8F8D14DC8FE194E010DC88A110
:103650000FDC83E294E00BDC89A10ADCCE01DF9170
:10366000CF9196CEF7DAD6CF87E294E000DCF2DA9B
:1036700038DBF0DACFDF77DA70E060E088E090E006
:10368000AFDE71DA70E060E089E090E0A9DE6BDA2D
:1036900070E060E08AE090E0A3DE65DA70E060E070
:1036A0008DE090E09DDE90E080E008954F925F9283
:1036B0006F927F928F929F92AF92BF92CF92DF9242
:1036C000EF92FF920F931F93CF936B017C01742EA7
:1036D000AC019B010E949C60882391F08EE294E0F3
:1036E000CF911F910F91FF90EF90DF90CF90BF90FF
:1036F000AF909F908F907F906F905F904F903ACB5C
:1037000046015701E894B7F82FEF3FEF4FE75FE727
:10371000C501B4010E949C6081110DC02FEF3FEFE5
:103720004FE75FE7C501B4010E940B5E18161CF459
:1037300082E394E0D5CF2FEF3FEF4FE75FE4C7017F
:10374000B6010E94986018161CF486E394E0C8CF76
:103750002FEF3FEF4FE75FECC701B6010E940B5E12
:1037600087FDF3CF20E030E0A901C701B6010E9438
:103770000B5E10E000E087FF08C08DE20E94840825
:103780008C01F7FAF094F7F8F094C0E060E070E094
:1037900080E09FE37C1641F020E030E040E251E41D
:1037A0000E94FF5FCF5FF6CFA70196010E949B5F4B
:1037B0002B013C010E946C604B015C014AE0E7DA9E
:1037C0007C01E00EF11ECC23A9F1C501B4010E94D9
:1037D0000F5E9B01AC01C301B2010E949A5F4B01D5
:1037E0005C018EE20E948408E80EF91EC15010F1BF
:1037F00020E030E040E251E4C501B4010E94705E77
:103800002B013C010E946C604B01B12CA12C4AE0C1
:10381000C501B401BCDAE80EF91EC501B4010E946D
:103820000F5E9B01AC01C301B2010E949A5F4B0184
:103830005C01DCCFC701CF911F910F91FF90EF90FA
:10384000DF90CF90BF90AF909F908F907F906F90C0
:103850005F904F9008958F929F92AF92BF92CF92B8
:10386000DF92EF92FF920F931F93CF93DF93EC01C0
:103870008AE392E0FCDA8FE494E0F9DA6E018EE2FA
:10388000C81A8EEFD80AC6010E94370D0E94115E39
:103890004B015C01FE01E151FD4F6081718182812C
:1038A00093810E94115E9B01AC01C501B4010E948D
:1038B000FF5F42E0FBDE8FE594E0D9DA7E01E2E0D3
:1038C000EE0EFE1EC7010E94370D0E94115E4B01D5
:1038D0005C01FE01ED50FD4F608171818281938119
:1038E0000E94115E9B01AC01C501B4010E94FF5F03
:1038F00042E0DCDE8FE694E0BADA8E010E5C1D4F0A
:10390000C8010E94370D0E94115E4B015C01C95035
:10391000DD4F688179818A819B810E94115E9B01C4
:10392000AC01C501B4010E94FF5F42E0BFDE92D945
:103930002FDD86E392E09BDA8FE494E098DAF601DB
:10394000A68DB78D20893189428953890E94635F92
:1039500061DA8FE594E08BDAF701A68DB78D2089C7
:103960003189428953890E94635F54DA8FE694E07B
:103970007EDAF801A68DB78D208931894289538975
:103980000E94635F47DA66D9DF91CF911F910F9153
:10399000FF90EF90DF90CF90BF90AF909F908F906F
:1039A000F7CCCF92DF92EF92FF92CF93DF93EC01AF
:1039B00088819981AA81BB81181619061A061B06EF
:1039C00044F081E090E0A0E0B0E088839983AA838E
:1039D000BB838C819D81AE81BF81181619061A06A2
:1039E0001B0644F081E090E0A0E0B0E08C839D8372
:1039F000AE83BF8388859985AA85BB85181619066D
:103A00001A061B0644F081E090E0A0E0B0E0888751
:103A10009987AA87BB878AE394E029DA8FE494E048
:103A200026DA6E857F85888999890E94115E6B01EF
:103A30007C01688179818A819B810E94115E9B0152
:103A4000AC01C701B6010E94FF5F42E02FDE8FE5A7
:103A500094E00DDA6A897B898C899D890E94115EC8
:103A60006B017C016C817D818E819F810E94115E42
:103A70009B01AC01C701B6010E94FF5F42E016DE68
:103A80008FE694E0F4D96E897F89888D998D0E94A4
:103A9000115E6B017C01688579858A859B850E9412
:103AA000115E9B01AC01C701B6010E94FF5F42E0BD
:103AB000FDDDCE01DF91CF91FF90EF90DF90CF90B1
:103AC00067CCC8D86EDF90E080E00895FC0180816B
:103AD0009181009711F00C942E5908950C942E5951
:103AE0000C942E590C942E590C942E590C942E593A
:103AF0000C942E590C942E590C942E590C942E592A
:103B00000C942E590C942E590C942E590C942E5919
:103B10000C942E590C942E590C942E590C942E5909
:103B20000C942E590C942E590C942E590C942E59F9
:103B30000C942E590C942E59CF92DF92EF92FF9253
:103B40000F931F93CF93DF938C016A017B01EC01EC
:103B5000CC0FDD1F642FCE010E942F5F9927F7FC49
:103B60009A958F2D7E2D6D2DCE0101960E942F5F8F
:103B70000D5811090330110588F4B701992777FD15
:103B80009095892FCE0144960E942F5F6F2D772745
:103B900088279927CE0145960E942F5F90E080E00C
:103BA000DF91CF911F910F91FF90EF90DF90CF9019
:103BB00008954F925F926F927F928F929F92AF92F1
:103BC000BF92CF92DF92EF92FF920F931F93CF930A
:103BD000DF938C01EC01CC0FDD1FCE010E94275F2B
:103BE000882E912CB12CA12CCE0101960E94275F2A
:103BF000C82ED12CF12CE12C0D58110903301105E0
:103C000008F05AC0CE0144960E94275F482E512CDE
:103C1000712C612CCE0145960E94275F082F10E081
:103C200030E020E08FEF481651046104710429F55B
:103C30000F3F11052105310501F58FEF881691041D
:103C4000A104B104C9F58FEFC816D104E104F10451
:103C500099F56FEF7FEFCB01DF91CF911F910F911E
:103C6000FF90EF90DF90CF90BF90AF909F908F909C
:103C70007F906F905F904F90089500381105210557
:103C800031053CF7FE2CED2CDC2CCC24C701B60111
:103C9000680D791D8A1D9B1D320155244424640D35
:103CA000751D861D971D302F222711270027600FB5
:103CB000711F821F931FD0CF00E010E09801412CAC
:103CC000512C320180E8C816D104E104F104D4F289
:103CD000C0CFEF92FF920F931F93CF93DF9380910A
:103CE000670890916808892B51F586E090E00E9462
:103CF00092587C0190E080E05CDF1616170654F1C4
:103D0000C7010E941F0DD0E0C0E0CE010E9406074F
:103D1000882369F0FE01EE0FFF1FEE0FFF1FE9572A
:103D2000F64F4081518162817381CE0105DF21967A
:103D3000C639D10551F7F0926808E0926708809182
:103D4000670890916808DF91CF911F910F91FF90C4
:103D5000EF90089583E090E02CDF613071058105DC
:103D6000910531F507E819E0D0E0C0E0CE010E94EE
:103D700006078823B1F0CE011CDFF8016083718350
:103D8000828393836F3F7F4F8F4F9F4F51F4CE01BC
:103D90000E94D401F8014081518162817381CE017A
:103DA000CBDE21960C5F1F4FC13ED105F9F6C3CF84
:103DB000C7010E941F0DBFCFCF92DF92EF92FF92FB
:103DC0000F931F93CF93DF937C016B018A01E9016D
:103DD00080DFF601EE0FFF1FEE0FFF1FE957F64FD2
:103DE00080819181F7019183808373DF000F111F20
:103DF000000F111FF801E957F64F81E04081518112
:103E000062817381413051056105710509F080E0DF
:103E1000F70182875EDFCC0FDD1FCC0FDD1FC95796
:103E2000D64F88819981AA81BB81F70182839383D0
:103E3000A483B5831682178210861186DF91CF91F5
:103E40001F910F91FF90EF90DF90CF900895CF9347
:103E5000DF93EC012AEC30E04BEC50E069EC70E0D1
:103E6000ABDF2EEC30E04FEC50E06DEC70E0CE01BB
:103E70000C96A2DF24ED30E045ED50E063ED70E0FC
:103E8000CE01489699DF28ED30E049ED50E067ED2E
:103E900070E0CE01849690DF2EED30E04FED50E0E3
:103EA0006DED70E0CE01C096DF91CF9185CFCF93BD
:103EB000DF9380916B0890916C08892BA1F48CE3BF
:103EC00090E00E949258EC01198218821D861C868F
:103ED000198E188E1DA21CA219AA18AAB8DFD09399
:103EE0006C08C0936B0880916B0890916C08DF910F
:103EF000CF9108952F923F924F925F926F927F924F
:103F00008F929F92AF92BF92CF92DF92EF92FF92E9
:103F10000F931F93CF93DF93EC01DBDEFE01EB5D8C
:103F2000FC4F8091430B9091440B91838083D1DEB1
:103F3000FE01E95DFC4F8091470B9091480B918306
:103F40008083C7DEFE01E75DFC4F80914B0B9091B3
:103F50004C0B91838083BDDE8E01055D1C4F60910B
:103F60006B0B70916C0B80916D0B90916E0B0E949E
:103F7000115EF8016083718382839383AADE1E0140
:103F8000F1ED2F1AFCEF3F0A60916F0B7091700BEF
:103F90008091710B9091720B0E94115EF101608310
:103FA00071838283938395DE20E030E048EC52E415
:103FB000F80160817181828193810E94FF5F2B01F2
:103FC0003C0120E030E048EC52E4F1016081718175
:103FD000828193810E94FF5F4B015C016091730BB2
:103FE0007091740B8091750B9091760B0E94115E0D
:103FF00020E030E048EC52E40E94FF5F6B017C015E
:104000002AE037ED43E25CE3C301B2010E9498600D
:1040100018160CF02BC120E030E046EC52E4C3014E
:10402000B2010E940B5E87FD06C0412C512C56EC5C
:10403000652E52E4752EF8014082518262827382AD
:104040002AE037ED43E25CE3C501B4010E949860C9
:1040500018160CF014C120E030E046EC52E4C50123
:10406000B4010E940B5E87FD06C0812C912C36ECBA
:10407000A32E32E4B32EF10180829182A282B38218
:104080002AE037ED43E25CE3C701B6010E94986085
:1040900018160CF0FDC020E030E046EC52E4C701F9
:1040A000B6010E940B5E87FD06C0C12CD12C96EC98
:1040B000E92E92E4F92EFE01ED5CFC4FC082D18224
:1040C000E282F38206DE80912B0B90912C0BFE0195
:1040D000E65CFC4F91838083FCDD80912F0B9091F7
:1040E000300BFE01E45CFC4F91838083F2DD809114
:1040F000330B9091340BFE01E25CFC4F9183808383
:10410000E8DD8091530B9091540BA091550BB09129
:10411000560BFE01E05CFC4F80839183A283B38346
:10412000D8DD8091570B9091580BA091590BB0910D
:104130005A0BFE01EC5BFC4F80839183A283B38317
:10414000C8DD80915B0B90915C0BA0915D0BB091F1
:104150005E0BFE01E85BFC4F80839183A283B383F7
:10416000B8DD80917B0B90917C0BFE01E45BFC4FF2
:1041700091838083AEDD80917F0B9091800BFE0157
:10418000E25BFC4F91838083A4DD8091830B90914F
:10419000840BFE01E05BFC4F918380839ADD80916C
:1041A000930B9091940BFE01EE5AFC4F9183808308
:1041B00090DD8091970B9091980BFE01EC5AFC4F8B
:1041C0009183808386DD80919B0B90919C0BFE01F7
:1041D000EA5AFC4F918380837CDD80911B0B909188
:1041E0001C0BA0911D0BB0911E0BFE01E95CFC4F56
:1041F0000197A105B10509F054C081E0808369DD14
:1042000080911F0B9091200BA091210BB091220B5C
:10421000FE01E85CFC4F0197A105B10509F043C020
:1042200081E0808356DD8091230B9091240BA09137
:10423000250BB091260BC75CDC4F0197A105B1059A
:10424000A1F581E08883DF91CF911F910F91FF90BD
:10425000EF90DF90CF90BF90AF909F908F907F9026
:104260006F905F904F903F902F9008954AE0442EBA
:1042700047ED542E43E2642E4CE3742EDCCE2AE04C
:10428000822E27ED922E23E2A22E2CE3B22EF3CE25
:104290008AE0C82E87EDD82E83E2E82E8CE3F82E34
:1042A0000ACF1082ACCF1082BDCF1882CCCF2F9214
:1042B0003F924F925F926F927F928F929F92AF92B6
:1042C000BF92CF92DF92EF92FF920F931F93CF9303
:1042D000DF93CDB7DEB765970FB6F894DEBF0FBE9C
:1042E000CDBF998B888BF5DCE889F989E358FD4FC0
:1042F00081E04091530A5091540A6091550A70919F
:10430000560A452B462B472B09F480E08083E1DCDD
:10431000E889F989E258FD4F81E04091570A5091B0
:10432000580A6091590A70915A0A452B462B472B1F
:1043300009F480E08083CDDCE889F989E158FD4FFC
:1043400081E040915B0A50915C0A60915D0A709136
:104350005E0A452B462B472B09F480E08083B9DCAD
:104360008091A30A9091A40AA091A50AB091A60AEF
:10437000E889F989E058FD4F80839183A283B38354
:10438000A8DC8091A70A9091A80AA091A90AB091EF
:10439000AA0AE889F989EC57FD4F80839183A283AB
:1043A000B38397DC8091AB0A9091AC0AA091AD0ADF
:1043B000B091AE0AE889F989E857FD4F808391836F
:1043C000A283B38386DC80917B0A90917C0AA091C2
:1043D0007D0AB0917E0AE889F989E856FD4F80830D
:1043E0009183A283B38375DC80917F0A9091800AC8
:1043F000A091810AB091820AE889F989E456FD4FBB
:1044000080839183A283B38364DC8091830A90913B
:10441000840AA091850AB091860AE889F989E05654
:10442000FD4F80839183A283B38353DC80918B0AF9
:1044300090918C0AA0918D0AB0918E0AE889F98931
:10444000EC55FD4F80839183A283B38342DC80913E
:104450008F0A9091900AA091910AB091920AE889EE
:10446000F989E855FD4F80839183A283B38331DCC2
:104470008091930A9091940AA091950AB091960A1E
:10448000E889F989E455FD4F80839183A283B38342
:1044900020DC80912B0A90912C0AA0912D0AB091DA
:1044A0002E0AE889F989E055FD4F80839183A28324
:1044B000B3830FDC80912F0A9091300AA091310ACA
:1044C000B091320AE889F989EC54FD4F80839183D9
:1044D000A283B383FEDB8091330A9091340AA091CA
:1044E000350AB091360AE889F989E854FD4F80838E
:1044F0009183A283B383EDDBE889F989E454FD4F0E
:1045000081E02091030A3091040A2130310509F03D
:1045100080E08083DEDBE889F989E354FD4F81E0A8
:104520002091070A3091080A2130310509F080E016
:104530008083CFDBE889F989E254FD4F81E0209147
:104540000B0A30910C0A2130310509F080E080839C
:10455000C0DBE889F989E652FD4F81E04091DB0933
:104560005091DC096091DD097091DE09452B462BE5
:10457000472B09F480E08083ACDBE889F989E552B8
:10458000FD4F81E04091DF095091E0096091E10920
:104590007091E209452B462B472B09F480E080837C
:1045A00098DBE889F989E452FD4F81E04091E30905
:1045B0005091E4096091E5097091E609452B462B7D
:1045C000472B09F480E0808384DBE889F989E35292
:1045D000FD4F81E04091B30A5091B40A6091B50A51
:1045E0007091B60A452B462B472B09F480E0808357
:1045F00070DBE889F989E252FD4F81E04091B70A0A
:104600005091B80A6091B90A7091BA0A452B462BAD
:10461000472B09F480E080835CDBE889F989E1526B
:10462000FD4F81E04091BB0A5091BC0A6091BD0AE8
:104630007091BE0A452B462B472B09F480E08083FE
:1046400048DBE889F989E052FD4F81E02091EB09D0
:104650003091EC092130310509F080E0808339DBAD
:10466000E889F989EF51FD4F81E02091EF09309100
:10467000F0092130310509F080E080832ADBE889E8
:10468000F989EE51FD4F81E02091F3093091F40951
:104690002130310509F080E080831BDB8091B30974
:1046A0009091B409A091B509B091B609E889F9894A
:1046B000ED51FD4F80839183A283B3830ADB809108
:1046C000B7099091B809A091B909B091BA09E889E0
:1046D000F989E951FD4F80839183A283B383F9DA8D
:1046E0008091BB099091BC09A091BD09B091BE0910
:1046F000E889F989E551FD4F80839183A283B383D3
:10470000E8DAE889F989E253FD4F81E04091C30975
:104710005091C4096091C5097091C609452B462B7B
:10472000472B09F480E08083D4DAE889F989E153E2
:10473000FD4F81E04091C7095091C8096091C909B6
:104740007091CA09452B462B472B09F480E08083E2
:10475000C0DAE889F989E053FD4F81E04091CB0947
:104760005091CC096091CD097091CE09452B462B13
:10477000472B09F480E08083ACDA8091BB0B9091E9
:10478000BC0BA091BD0BB091BE0BE889F989E15437
:10479000FD4F80839183A283B3839BDA8091BF0B0B
:1047A0009091C00BA091C10BB091C20BE889F9891F
:1047B000ED53FD4F80839183A283B3838ADA809186
:1047C000C30B9091C40BA091C50BB091C60BE889A7
:1047D000F989E953FD4F80839183A283B38379DA0A
:1047E000E889F989EF52FD4F81E020911B0A309151
:1047F0001C0A2130310509F080E08083E889F989BD
:10480000EE52FD4F1082E889F989ED52FD4F10827A
:1048100060DAE889F989EC52FD4F81E02091170AAE
:104820003091180A2130310509F080E08083E88951
:10483000F989EB52FD4F1082E889F989EA52FD4F60
:10484000108247DAE889F989E952FD4F81E0209129
:104850003B0A30913C0A2130310509F080E0808329
:1048600038DAE889F989E852FD4F81E020913F0A62
:104870003091400A2130310509F080E0808329DA47
:10488000E889F989E752FD4F81E02091430A309190
:10489000440A2130310509F080E080831ADAE88982
:1048A000F989E553FD4F81E02091CB0B3091CC0B82
:1048B0002130310509F080E080830BDAE889F9893D
:1048C000E453FD4F81E02091CF0B3091D00B21308C
:1048D000310509F080E08083FCD9E889F989E35348
:1048E000FD4F81E02091D30B3091D40B2130310565
:1048F00009F080E08083EDD90889198901511D4FA5
:104900008091630A9091640AA091650AB091660A49
:10491000F80180839183A283B383DBD9E888F98887
:10492000FDE0EF1AFDEFFF0A8091670A9091680A97
:10493000A091690AB0916A0AF70180839183A283EA
:10494000B383C7D980916B0A90916C0AA0916D0ACC
:10495000B0916E0AC888D988F9E0CF1AFDEFDF0A56
:10496000F60180839183A283B383F8014081518152
:1049700062817381141615061606170644F041E08D
:1049800050E060E070E04083518362837383F701FD
:10499000408151816281738114161506160617062F
:1049A00044F041E050E060E070E040835183628376
:1049B0007383181619061A061B064CF081E090E066
:1049C000A0E0B0E0F60180839183A283B3830E94CC
:1049D0002A16FC01D6018D909D90AD90BC90D70118
:1049E0004D915D916D917C91D8010D911D912D910D
:1049F0003C910083118322833383448355836683F0
:104A0000778380869186A286B386E889F989709635
:104A1000FB83EA83E889F989E553FD4F20812983E7
:104A2000E889F989E154FD4F80819181A281B381A8
:104A3000E889F989E952FD4F20812A87E889F989B7
:104A4000E052FD4F20812C83E889F989EF52FD4F18
:104A500020812D83E889F989EC52FD4F20812E8336
:104A6000E889F989E352FD4F20812E87E889F98989
:104A7000E652FD4F20812F87E889F989E454FD4FE4
:104A80002080E889F989E358FD4F3080E889F98969
:104A9000ED51FD4F4081518162817381E889F9892F
:104AA000E055FD4F0081118122813381E889F98928
:104AB000EC55FD4FC080D180E280F380E889F98910
:104AC000E856FD4F80809180A280B380E889F98903
:104AD000E058FD4F4080518062807380E889F989F9
:104AE00044AE55AE66AE77AEE05CFF4F80829182F9
:104AF000A282B382E889F989EC5BFF4FC082D18240
:104B0000E282F382E889F989E85BFF4F0083118331
:104B100022833383E889F989E45BFF4F4083518323
:104B200062837383E889F989E05BFF4F3082E8890B
:104B3000F989EF5AFF4F20822F85E889F98921AF43
:104B40002E8522AF2C8123AF40E450E060E070E07E
:104B5000EC5AFF4F4083518362837383E889F9895C
:104B6000EE5AFF4F2E812083E889F989ED5AFF4FD5
:104B70002D812083E889F989E85AFF4F2A8520830F
:104B8000E889F989E75AFF4F80839183A283B38331
:104B9000E889F989E35AFF4F89818083A889B98917
:104BA00099968D919C919A978633910509F083C2CD
:104BB00080E091E1FD01EA56FF4F918380833296B8
:104BC0001182108282E091E1369691838083329641
:104BD00011821082E889F98987A590A94A97D1F4B2
:104BE00084E191E1E656FF4F91838083E889F9895A
:104BF000E456FF4F1182108286E191E1E889F9893C
:104C0000EE55FF4F91838083E889F989EC55FF4F7A
:104C100011821082088919890A551F4FE889F9897C
:104C2000E453FD4F20812983E889F989ED53FD4F35
:104C300080819181A281B3818A879B87AC87BD8760
:104C4000E889F989E852FD4F90819C83E889F989C8
:104C5000EF51FD4FA081AD83E889F989EE52FD4FF8
:104C6000B081BE83E889F989EB52FD4F20812E8700
:104C7000E889F989E252FD4F2080E889F989E552F7
:104C8000FD4F3080E889F989E354FD4F3081E88990
:104C9000F989E258FD4F2081E889F989E951FD4FF2
:104CA00080819181A281B381E889F989EC54FD4F1B
:104CB0004081518162817381E889F989E855FD4F0E
:104CC000C080D180E280F380E889F989E456FD4F05
:104CD00080809180A280B380E889F989EC57FD4FEC
:104CE0004080518062807380F80144A655A666A674
:104CF00077A680AA91AAA2AAB3AAC4AAD5AAE6AA0C
:104D0000F7AA40AF51AF62AF73AF84AF95AFA6AF14
:104D1000B7AFE889F989EA51FF4F2083E889F9891B
:104D2000E951FF4F3083D80199963C9299979A9612
:104D30002C929A97ED819B96EC9380E490E0A0E012
:104D4000B0E0E889F989E651FF4F80839183A2831F
:104D5000B383E889F989E851FF4F2E852083E889DC
:104D6000F989E751FF4F8E818083E889F989E25103
:104D7000FF4F9C819083E889F989E151FF4F8A8533
:104D80009B85AC85BD8580839183A283B383E889AD
:104D9000F989ED50FF4F99819083D80159968D91F3
:104DA0009C918633910509F0B8C180E091E1E889D2
:104DB000F989E45DFE4F91838083E889F989E25D9A
:104DC000FE4F1182108282E091E1E889F989EC5C62
:104DD000FE4F91838083E889F989EA5CFE4F118256
:104DE0001082F801878D90A14A97E1F484E191E166
:104DF000E889F989E05DFE4F91838083E889F9892C
:104E0000EE5CFE4F1182108286E191E1E889F9891A
:104E1000E85CFE4F91838083E889F989E65CFE4F68
:104E200011821082E888F988F4ECEF1AFEEFFF0A8D
:104E3000E889F989E353FD4F20812983E889F989BD
:104E4000E953FD4F80819181A281B3818A879B873D
:104E5000AC87BD87E889F989E752FD4F90819C8333
:104E6000E889F989EE51FD4F3080E889F989ED52E2
:104E7000FD4FA081AD83E889F989EA52FD4F20807A
:104E8000E889F989E152FD4FC080E889F989E45247
:104E9000FD4FD080E889F989E254FD4F3081E889DF
:104EA000F989E158FD4F2081E889F989E551FD4FE5
:104EB00080819181A281B3818A8B9B8BAC8BBD8BCE
:104EC000E889F989E854FD4F4081518162817381FD
:104ED000E889F989E455FD4F80809180A280B380F4
:104EE000E889F989E056FD4F4080518062807380E7
:104EF000E889F989E857FD4F80819181A281B381CA
:104F0000F70184A795A7A6A7B7A740AA51AA62AAA6
:104F100073AA84AA95AAA6AAB7AA40AF51AF62AF56
:104F200073AF8A899B89AC89BD8984AF95AFA6AFE1
:104F3000B7AFE889F989E458FE4F2083E889F989F9
:104F4000E358FE4F3083D7019996DC9299979A9651
:104F5000CC929A979B963C9280E490E0A0E0B0E0DF
:104F6000E889F989E058FE4F80839183A283B38357
:104F7000E889F989E258FE4F2082E889F989E158E9
:104F8000FE4FBD81B083E889F989EC57FE4F2C8133
:104F90002083E889F989EB57FE4F8A859B85AC858C
:104FA000BD8580839183A283B383E889F989E7571C
:104FB000FE4F99819083D70159968D919C918633AC
:104FC000910509F0D2C080E091E1E889F989EE53BA
:104FD000FE4F91838083E889F989EC53FE4F11825B
:104FE000108282E091E1E889F989E653FE4F9183CE
:104FF0008083E889F989E453FE4F11821082F7011A
:10500000878D90A14A97E1F484E191E1E889F989DB
:10501000EA53FE4F91838083E889F989E853FE4F74
:105020001182108286E191E1E889F989E253FE4F0D
:1050300091838083E889F989E053FE4F11821082C1
:10504000E889F989E253FD4F8081882309F4B5C0CE
:105050008A819B810E94E211E889F989E153FD4F21
:105060008081882309F4AEC0C8010E94E2118889BA
:10507000998980539D4FDC018C91882309F4A6C047
:10508000C70165960FB6F894DEBF0FBECDBFDF91A6
:10509000CF911F910F91FF90EF90DF90CF90BF9035
:1050A000AF909F908F907F906F905F904F903F90C8
:1050B0002F900C94E2118C339105D9F484E091E1A6
:1050C000E889F989EA56FF4F91838083E889F98955
:1050D000E856FF4F1182108286E091E1E889F98954
:1050E000E256FF4F91838083E889F989E056FF4FAC
:1050F0006FCD8E9709F06ECD88E091E1E889F9894E
:10510000EA56FF4F91838083E889F989E856FF4F7B
:10511000118210828EE091E1E1CF8C33910589F408
:1051200084E091E1E889F989E45DFE4F9183808311
:10513000E889F989E25DFE4F1182108286E091E1F3
:1051400044CE8E9709F04DCE88E091E1E889F98947
:10515000E45DFE4F91838083E889F989E25DFE4F2B
:10516000118210828EE091E130CE8C33910589F46A
:1051700084E091E1E889F989EE53FE4F91838083C1
:10518000E889F989EC53FE4F1182108286E091E1A3
:105190002ACF8E9709F033CF88E091E1E889F98929
:1051A000EE53FE4F91838083E889F989EC53FE4FDB
:1051B000118210828EE091E116CF8A819B810E943C
:1051C000A1114ACFC8010E94A11151CFC701659614
:1051D0000FB6F894DEBF0FBECDBFDF91CF911F9108
:1051E0000F91FF90EF90DF90CF90BF90AF909F9086
:1051F0008F907F906F905F904F903F902F900C9486
:10520000A111AF92BF92CF92DF92EF92FF920F93D4
:105210001F93CF93DF93EC018AE190E09AA789A7CF
:105220008BE190E09CA78BA789E190E09EA78DA7DA
:105230008FE090E098AB8FA78EE190E09AAB89ABBE
:105240008EE090E09CAB8BAB85E490E09EAB8DABA9
:1052500084E490E098AF8FABFE01EA55FF4F80E207
:1052600090E0928F818F81E290E0948F838F8FE125
:1052700090E0968F858F10A2178E12A211A214A211
:1052800013A283E490E096A385A382E490E090A724
:1052900087A3EA56FF4F83E290E0928F818F84E2EA
:1052A00090E0948F838F82E290E0968F858F10A29A
:1052B000178E12A211A214A213A281E490E096A369
:1052C00085A380E490E090A787A3E55CFE4F118260
:1052D0001082329611821082329611821082CE0193
:1052E0000E945721CE010E947A1FCE018E529E4FFE
:1052F00041E050E0FC0157A746A7DE01AE5FBD4F7D
:1053000024E030E09F963C932E939E975E01FEEC46
:10531000AF1AFDEFBF0A28E030E0F50137A726A756
:1053200020E130E0FC013183208321E130E035834E
:1053300024832FEF3FEF33832283378326836285D5
:1053400060876385618767E170E011967C936E9357
:1053500068E170E015967C936E93149713963C93D6
:105360002E93129717963C932E9316971A966C913C
:105370001A9718966C9318971B966C911B97199611
:105380006C9319976DE170E0F501718360836CE1B6
:1053900070E0758364833383228337832683628539
:1053A000608763856187BE016E5A7C4FFB01608117
:1053B00071818E01005C1C4FF801C080D180E280B9
:1053C000F38006501109F80100811181FC01158F4D
:1053D000048FC48AD58AE68AF78A6130710509F09C
:1053E0004EC0378F268FCE018C5A9C4FFC01808196
:1053F00091819E012C5B3C4FF9014081518162817A
:10540000738128503109F901208131815D963C93E7
:105410002E935C9754964D935D936D937C93579721
:10542000019781F58FEF9FEF5F969C938E935E9728
:10543000DE01AA5ABC4F8D919C9111971E974D91F8
:105440005D916D917C91C25CDC4F28813981F501C1
:10545000358F248F448B558B668B778B0197A9F4FE
:105460008FEF9FEF978F868FDF91CF911F910F91D5
:10547000FF90EF90DF90CF90BF90AF900895578F3F
:10548000468FB1CF81E090E0CFCF81E090E0EACFCE
:10549000EF92FF920F931F93CF93DF93EC010E9443
:1054A000691E0091D30A1091D40A0E94691EE090EF
:1054B000E30AF090E40A0E94691E2091FB0A3091F1
:1054C000FC0A1216130614F021E030E0A701B8011F
:1054D000CE01845C9E4FDF91CF911F910F91FF9081
:1054E000EF900C94E413EF92FF920F931F93CF93DE
:1054F000DF93EC010E94691E0091CF0A1091D00A3F
:105500000E94691EE090DF0AF090E00A0E94691E86
:105510002091F70A3091F80A1216130614F021E0D0
:1055200030E0A701B801CE018A559F4FDF91CF919E
:105530001F910F91FF90EF900C94E413EF92FF9264
:105540000F931F93CF93DF93EC010E94691E00918C
:10555000CB0A1091CC0A0E94691EE090DB0AF09001
:10556000DC0A0E94691E2091F30A3091F40A121697
:10557000130614F021E030E0A701B801CE014096F7
:10558000DF91CF911F910F91FF90EF900C94E41356
:105590008F929F92AF92BF92CF92DF92EF92FF9243
:1055A000CF93DF937B010E94691EEC01F70182A07B
:1055B00093A0A4A0B5A0C68CD78CE0A0F1A08A814E
:1055C0009B818F30F7E29F070CF043C001969B83CD
:1055D0008A838C819D818F3027E29207ECF59601BA
:1055E0002B7F215531092330310530F096012B55A1
:1055F00031092330310518F401969D838C83C6014F
:105600000E940607882359F1F601EE0FFF1FEE0FE7
:10561000FF1FE957F64F80829182A282B382B501C3
:10562000A401C6010E949C1DB601CE010E94A71ACA
:105630000E94571F0E94271F90E080E0DF91CF91CA
:10564000FF90EF90DF90CF90BF90AF909F908F90A2
:1056500008951B821A82BDCF1D821C82D0CF8AED95
:1056600093E00E943717E4CFCF93DF93EB010E94C2
:10567000691E6E8D7F8D0E94A71A90E080E0DF91F9
:10568000CF9108950E94691E0E94E11A8EE394E072
:105690000E9437170E942A160E94C81990E080E0E5
:1056A00008950F931F93CF93DF93EC018881998125
:1056B000009759F02A813B812617370730F081E0A7
:1056C000DF91CF911F910F9108958B016F5F7F4FF5
:1056D0000E94EA60009759F0998388831B830A83AC
:1056E0002C813D81232B59F7FC011082E8CF80E00B
:1056F000E7CF0F931F93CF93DF93EC018B01D1DFA3
:1057000028813981811112C02115310519F0C90193
:105710000E942E59198218821D821C821B821A82B5
:10572000CE01DF91CF911F910F9108951D830C83BE
:1057300060E378E0C9010E94DC61F2CF70E060E0D4
:10574000D8CF2F923F924F925F926F927F928F921B
:105750009F92AF92BF92CF92DF92EF92FF920F9300
:105760001F93CF93DF93CDB7DEB7C659D1090FB6DC
:10577000F894DEBF0FBECDBF8C01FC0110821182F8
:105780001282138214821582168217821086118665
:105790001286138614861586168617864C01F0E14C
:1057A0008F0E911CC4010E945A14580186EAA80E5B
:1057B000B11CC5010E945A146801E4ECCE1AEEEF48
:1057C000DE0AC6010E945A147801FEE2EF1AFEEFCB
:1057D000FF0AC7010E94990D380182E0680E781E09
:1057E000C3010E94990D2801EEEC4E1AEDEF5E0AFE
:1057F000C2010E94990DF801EE59FD4F11821082ED
:105800001382128215821482CF0198DFF801E859C1
:10581000FD4F1182108232961182108232961182CF
:105820001082329611821082329610821182128278
:1058300013823496108231961082319610823196FE
:105840001182108232961182108232961182108259
:1058500032961082319610823196108231961082E3
:105860001182128213823496108211821282138264
:105870003496108211821282138234961082118221
:10588000128213823496108211821282138234960D
:105890001082118212821382349610821182128237
:1058A00013823496108211821282138234961082EF
:1058B0001182128213823496108211821282138214
:1058C00034961082118212821382349610821182D1
:1058D00012821382349610821182128213823496BD
:1058E00010821182128213823496108211821282E7
:1058F000138234961082319610823196108231963E
:1059000010821182128213823496108211821282C6
:10591000138234961082118212821382349610827E
:105920003196108231961082319610823196108213
:105930003196108231961082319610823196108203
:1059400031961082319610823196108231961082F3
:1059500031961082319610823196108231961082E3
:1059600031961082319610823196108231961082D3
:1059700031961082319610823196108231961082C3
:105980001182128213823496108211821282138243
:1059900034961082118212821382D801A151BD4F18
:1059A0008CE0E9E1F2E001900D928A95E1F7F801CF
:1059B000E550FD4F108211821282138234961082BC
:1059C0001182128213823496108211821282138203
:1059D0003496118210823296118210823296118290
:1059E00010823296108211821282138234961082B3
:1059F00011821282138234961082118212821382D3
:105A0000349610821182128213823496108211828F
:105A1000128213823496108211821282138234967B
:105A20001182108232961182108232961182108277
:105A30003296108211821282138234961082118261
:105A4000128213823496108211821282138234964B
:105A50001082319610823196108231961182108216
:105A60003296118210823296118210823296108202
:105A70001182128213823496108211821282138252
:105A8000349610821182128213823496118210820F
:105A900032961182108232961182108232961182D1
:105AA00010823296118210823296118210823296C2
:105AB000118210823296118210821801F4EA2F1A94
:105AC000FCEF3F0AF101108231961182108232966A
:105AD00011821082CE0101960E945A1486E9FE01BD
:105AE0003196D40101900D928A95E1F7CE0101968D
:105AF0000E945A1486E9FE013196D50101900D925B
:105B00008A95E1F7CE0101960E945A1486E9FE01BA
:105B10003196D60101900D928A95E1F788E5F8015A
:105B2000848BE655FF4F89E58083EA56FF4F8AE56F
:105B30008083CE0101960E94990D80E3FE0131968B
:105B4000D70101900D928A95E1F7CE0101960E944E
:105B5000990D80E3FE013196D30101900D928A9553
:105B6000E1F7CE0101960E94990D80E3FE01319686
:105B7000D20101900D928A95E1F7C80142DBF10153
:105B80001082CA56DF4F0FB6F894DEBF0FBECDBFEE
:105B9000DF91CF911F910F91FF90EF90DF90CF9009
:105BA000BF90AF909F908F907F906F905F904F903D
:105BB0003F902F900895CF93DF9380916508909147
:105BC0006608892B51F481E693E00E949258EC011B
:105BD000B8DDD0936608C093650880916508909100
:105BE0006608DF91CF910895CF93DF938091640889
:105BF000811121C081E080936408DDDFEC014096D3
:105C00000E94AE13CE018A559F4F0E94AE13CE0163
:105C1000845C9E4F0E94AE13C059DD4F88819981EC
:105C2000AA81BB810196A11DB11D88839983AA8396
:105C3000BB8310926408DF91CF910895CF93DF93D7
:105C4000EB0120E030E040E85FE36A817B818C81FA
:105C50009D810E940B5E811110C082E494E00E943D
:105C60003717A9DFFC01EE59FF4F10821182128213
:105C700013828E529E4F0E94CD0F20E030E040E80C
:105C80005FE36E817F81888599850E940B5E81111B
:105C900010C082E594E00E9437178DDFFC01E850C8
:105CA000FF4F10821182128213828E5F9D4F0E94DD
:105CB000CD0F20E030E040E85FE36A857B858C858E
:105CC0009D850E940B5E811110C082E694E00E94C7
:105CD000371771DFFC01E257FE4F108211821282EA
:105CE00013828E5C9D4F0E94CD0F0E942A160E9447
:105CF000C81990E080E0DF91CF910895CF93DF93B2
:105D0000FC01EA59FD4F408151814115510501F1D6
:105D1000EC01C659DD4F288139818E599D4F2417DA
:105D20003507E8F4FC01808191810097A1F0820F92
:105D3000931FFC0180818A3031F08D3069F48EE24E
:105D400098E00E943717888199810196998388830A
:105D5000DF91CF91089580E00E948408F4CF70E035
:105D600060E0C7DC19821882F3CFEF92FF920F93A5
:105D70001F93CF93DF936115710541F480E0DF91AC
:105D8000CF911F910F91FF90EF900895411551050C
:105D9000A9F07B01EC010C811D81040F151FB801D6
:105DA00080DC882359F3288139818C819D81B7015A
:105DB000820F931F0E94DC611D830C8381E0DFCF83
:105DC000EF92FF920F931F93CF93DF93CDB7DEB780
:105DD00064970FB6F894DEBF0FBECDBF7C01CB0138
:105DE000BA018E010F5F1F4F22E044E00E947558F8
:105DF000FC0101900020E9F73197AF01481B590BD6
:105E0000BC01C701B2DF64960FB6F894DEBF0FBEC7
:105E1000CDBFDF91CF911F910F91FF90EF9008952B
:105E2000EF92FF920F931F93CF93DF93CDB7DEB71F
:105E30002E970FB6F894DEBF0FBECDBF7C01CB010D
:105E4000BA012AE08E010F5F1F4FA8010E94EE5990
:105E5000F80101900020E9F73197AF01401B510B89
:105E6000B801C70182DF2E960FB6F894DEBF0FBED1
:105E7000CDBFDF91CF911F910F91FF90EF900895CB
:105E8000FB0101900020E9F73197AF01461B570B4A
:105E90006CCF0F931F93CF93DF93EC018B0119828B
:105EA00018821B821A821D821C8248DC6DEC73E012
:105EB000CE01E6DFF80142A153A164A175A1CE0194
:105EC000AFDF6EE278E0CE01DBDFCE01DF91CF9174
:105ED0001F910F910895FB0144815581608171816B
:105EE00044CFCF92DF92EF92FF920F931F93CF9305
:105EF000DF9300D000D01F921F92CDB7DEB78B0189
:105F00006A018E599D4F7C0162E372E0B9DF62E560
:105F100076E0C701B5DFF801848189831A8241E008
:105F200050E08E010F5F1F4FB801C7011EDF4AE02E
:105F3000B801C6010E94E459F80101900020E9F778
:105F40003197AF01401B510BB801C7010EDF0E9412
:105F50002A16BC01C8019DDFB801C701BCDFC8011A
:105F60000E94661D28960FB6F894DEBF0FBECDBF07
:105F7000DF91CF911F910F91FF90EF90DF90CF9025
:105F800008952F923F924F925F926F927F928F92DD
:105F90009F92AF92BF92CF92DF92EF92FF920F93B8
:105FA0001F93CF93DF93CDB7DEB7E3970FB6F89487
:105FB000DEBF0FBECDBF9BAB8AAB3B010E9457211A
:105FC0008AA99BA90E947A1F0E94250A4B015C01A5
:105FD0009301220F331F220F331F3A8329834AA9CB
:105FE0005BA9240F351F3F8B2E8B89010C551D4F4C
:105FF000D8016D917D918D919C910E94115E9B01C4
:10600000AC0160E074E284E796E40E94FF5F20E068
:1060100030E040E05FE30E94705E0E946C606A8B3B
:106020007B8B8C8B9D8B88E993E00E94371782E5F0
:1060300096E00E94371782E794E00E94371782E5C6
:1060400096E00E9437174AE06A897B898C899D898E
:106050000E94C71682E596E00E9437178DE794E00C
:106060000E94371782E596E00E94371780E490E09F
:106070000E94321782E596E00E94371786E994E085
:106080000E94371782E596E00E943717F801608179
:106090007181828193810E940A1782E596E00E94B5
:1060A00037178EE298E00E9437170E94B2160E94BE
:1060B000321B2AA83BA8F1E06F16710409F464C0F2
:1060C00022E06216710409F48EC030E1230E311C07
:1060D0004AA85BA84EE2441A4EEF540AEAA9FBA96B
:1060E000E652FD4F50815B878AA99BA985509D4F41
:1060F0009E838D83AAA9BBA9AB5DBC4FB98FA88F26
:10610000EAA9FBA9E95CFC4FFBA3EAA32AA93BA9E6
:1061100029583D4F3D872C874DE850E059A348A3AF
:1061200085E190E098878F83C1010E9451118823F7
:1061300009F48AC086EA94E00E9437170E942A1662
:1061400024E030E0DC0197963C932E93969734E060
:10615000632E712CC301E3960FB6F894DEBF0FBE19
:10616000CDBFDF91CF911F910F91FF90EF90DF9006
:10617000CF90BF90AF909F908F907F906F905F90E7
:106180004F903F902F90089596EA290E311C4AA80F
:106190005BA8A2E04A0E5A1EEAA9FBA9E552FD4FF0
:1061A000B081BB87EAA9FBA9E150FD4FFE83ED83D7
:1061B0002AA93BA9295D3C4F398F288F4AA95BA9A1
:1061C000485C5C4F5BA34AA38AA99BA987589D4F53
:1061D0009D878C87AEE8B0E0B9A3A8A3E6E1F0E024
:1061E000F887EF83A1CFF4EC2F1AFEEF3F0A4AA8FD
:1061F0005BA82EEC421A2DEF520AEAA9FBA9E45241
:10620000FD4F30813B874AA95BA94D5F5C4F5E83A0
:106210004D838AA99BA9875D9C4F998F888FAAA9D6
:10622000BBA9A75CBC4FBBA3AAA3EAA9FBA9E558DD
:10623000FD4FFD87EC872FE830E039A328A347E125
:1062400050E058874F8370CFC1010E9441118111E6
:1062500071CF88E993E00E9437178CED94E00E949B
:106260003717F10184810E94840883EE94E00E9434
:1062700037178EE298E00E94371781E090E0AC85F6
:10628000BD858D939C9341E050E0B1018AA99BA903
:1062900028DEC1010E94E211F101E05CFF4F808124
:1062A000810104581F4F882309F4D6C0C1010E9400
:1062B0006111F8011082C2010E94370DF101EE5AFE
:1062C000FF4F6083718382839383ED81FE8110820F
:1062D000118212821382EAA9FBA9E550FD4F1082B8
:1062E000118212821382EAA9FBA9E150FD4F1082AC
:1062F000118212821382EAA9FBA9ED5FFC4F108282
:1063000011821282138286E090E0AC85BD858D9368
:106310009C9346E050E0B1018AA99BA9E2DD61E0CF
:1063200070E0C1010E94D81989819A81855D9C4FD6
:10633000EAA9FBA9E80FF91FFDA3ECA3C3018A5545
:106340009E4F880F991F2AA93BA9280F391F3FA3E9
:106350002EA389819A81875E9C4F4AA95BA9480F29
:10636000591F59A748A789819A81835F9C4FAAA981
:10637000BBA9A80FB91FBBA7AAA789819A8185507D
:106380009D4FEAA9FBA9E80FF91FFDA7ECA71E8600
:106390001F86188A198A8AA99BA9860D971D9C01B8
:1063A000295C3C4F3FA72EA789819A814AA95BA906
:1063B000840F951FDC01AD51BD4FBB8FAA8F405993
:1063C0005D4F5F8F4E8FEE89FF89EC55FD4FF9AB26
:1063D000E8AB8AA99BA90E94E110AEA5BFA58C914C
:1063E000882371F0CCA0DDA0EEA0FFA008A519A520
:1063F0002AA53BA54CA55DA5B201C1010E942D10A7
:106400000E94250A681579058A059B0560F50E949A
:10641000250A681579058A059B0508F460C08CE09B
:106420009DE00E940108181619060CF46DC010E0DA
:106430001C821B82C1010E945111882309F485C06E
:1064400086E595E00E943717C1010E945111811124
:1064500001C08B858B871DC2C1010E94811181E023
:10646000D8018C9328CF0E94250A6B017C01C818A3
:10647000D908EA08FB08EA8DFB8D20813181428131
:106480005381A8EEB3E00E94595F6C157D058E051F
:106490009F0508F0BCCFC1010E94A111F1E06F1669
:1064A000710409F425C122E06216710409F4F9C0EF
:1064B00086E692E00E9437170E942A160E94C819A9
:1064C00082E095E00E9437170E942A1622E030E011
:1064D000FC0137A326A382E0682E712C3BCE0E94DC
:1064E000250A6B017C01AA8DBB8D2D913D914D91AB
:1064F0005C91A8EEB3E00E94595F6C157D058E0596
:106500009F0508F08CCFC7CF8CE09DE00E94DF078D
:106510008F7D8534910509F08ACF81E495E00E9452
:1065200037170E942A16E1E0DC01D496EC938AE545
:1065300092E00E9437170E942A160E94C81921E093
:1065400030E03C832B8311E075CFC1010E944111E3
:10655000811176CF111174CFA88DB98D6D917C9179
:10656000072E000C880B990B0E94115E9B01AC0159
:10657000ED81FE8160817181828193810E940B5E39
:1065800087FF5ECFC1010E949812AE8DBF8D4D91E5
:106590005D916D917C910A891B892C893D89040F3D
:1065A000151F261F371F401751076207730728F46E
:1065B00083EE93E00197F1F7F6CF2E853F8548896A
:1065C00059892F5F3F4F4F4F5F4F2E873F87488B33
:1065D000598BA8A9B9A92D913D914D915C91A3E04A
:1065E000B0E00E94595F9B01AC016E857F85888970
:1065F00099890E943D5F672B682B692B41F486E5E2
:1066000092E00E9437170E942A160E94C819C10101
:106610000E942811EE8DFF8D40815181628173812E
:106620000A891B892C893D89040F151F261F371FD6
:10663000401751076207730708F026C183EE93E005
:106640000197F1F7F5CFC1010E946111F8011082A5
:1066500094C10E94250A6B017C012F8138854985F0
:106660005A85C21AD30AE40AF50AA981BA812D9182
:106670003D914D915C91A8EEB3E00E94595F6C157D
:106680007D058E059F0508F0EDC1C1010E94A11195
:10669000B1E06B16710461F1E2E06E16710409F06D
:1066A00007CF8EE592E00E9437170E942A160E94BB
:1066B000C8198CE295E00E9437170E942A16FC0147
:1066C00077A266A247CD0E94250A6B017C01A981B1
:1066D000BA812D913D914D915C91A8EEB3E00E945D
:1066E000595F6C157D058E059F0508F0C7C1CDCF9C
:1066F00082E692E00E9437170E942A160E94C8196B
:1067000087E195E00E9437170E942A1622E030E0C8
:10671000DC0197963C932E939697DDCE8CE09DE01E
:106720000E94DF078F7D8534910509F0AFC181E4B8
:1067300095E00E9437170E942A16E1E0DC01D4960A
:10674000EC938AE592E00E9437170E942A160E9475
:10675000C81921E030E03C832B8311E098C111116E
:10676000ACC1E88DF98D60817181072E000C880B1A
:10677000990B0E94115E9B01AC01AD81BE816D91B0
:106780007D918D919C910E940B5E87FF96C1C10106
:106790000E949812BFEF8B1A9B0AAB0ABB0AEE85C8
:1067A000FF8540815181628173810A891B892C890F
:1067B0003D89040F151F261F371F40175107620719
:1067C000730728F483EE93E00197F1F7F6CFAE89D3
:1067D000BF892D913D914D915C91A3E0B0E00E9465
:1067E000595F9B01AC01C501B4010E943D5F672B5D
:1067F000682B692BC1F486E592E00E9437170E944E
:106800002A160E94C81988E993E00E94371785E983
:1068100095E00E943717C501B4010E940A178EE265
:1068200098E00E943717C1010E942811EE85FF856C
:1068300040815181628173810A891B892C893D893C
:10684000040F151F261F371F4017510762077307D4
:1068500008F0E0C083EE93E00197F1F7F5CF0E94D6
:106860002A16FC01828A938AA48AB58AA7C10E944B
:106870002A16DC0156968D929D92AD92BC92599744
:106880009DC10E94411116C12B813C81232B09F42B
:10689000A0CD62E070E0C1010E94D81988E993E0C0
:1068A0000E9437178CED94E00E943717D10114969F
:1068B0008C910E9484088AE695E00E9437178EE248
:1068C00098E00E943717EB81FC81EF2B09F58DE7EB
:1068D00095E00E94371782E596E00E94371784ED15
:1068E00093E00E9437178F8198850E94321782E5C6
:1068F00096E00E9437178FE598E00E943717FB85D6
:106900008F2F90E00E9432170E942A160E94C81909
:106910000E94B2160E94321B88E993E00E9437174A
:106920008CED94E00E943717D10114968C910E944F
:10693000840881E895E00E9437178EE298E00E9473
:1069400037170E94250A6F83788789879A87ED8198
:10695000FE811082118212821382F101E05CFF4FEE
:106960008081810104581F4F882309F46CCEC10136
:106970000E94811181E0D8018C93C2010E94370DE1
:10698000F101EE5AFF4F6083718382839383EAA9FA
:10699000FBA9E550FD4F1082118212821382EAA9F1
:1069A000FBA9E150FD4F1082118212821382EAA9E5
:1069B000FBA9ED5FFC4F1082118212821382C2018B
:1069C0000E94370D6A8F7B8F8C8F9D8FC2010E9432
:1069D000370D812C912C54018AA99BA9860D971DF6
:1069E0009C01295C3C4F3F8F2E8F89819A814AA957
:1069F0005BA9840F951FDC01AD51BD4FBA83A983FC
:106A000040595D4F5F874E87EE89FF89EC55FD4FFA
:106A1000FF8BEE8B2B813C81232B09F052C08AA97E
:106A20009BA90E94E110AE8DBF8D8C91882371F0DF
:106A3000CCA0DDA0EEA0FFA008A519A52AA53BA526
:106A40004CA55DA5B201C1010E942D100E94250A2E
:106A50002F81388549855A85621773078407950702
:106A600008F0F7CD0E94250A2F81388549855A857F
:106A7000621773078407950708F425CE8CE09DE024
:106A80000E940108181619060CF448CE10E03AE0EE
:106A900083169104A104B1043CF4AD81BE811D9222
:106AA0001D921D921C921397BB85C101B111E9CEB5
:106AB0000E945111882309F452CE86E595E00E9488
:106AC000371788E993E00E9437178CED94E00E9415
:106AD0003717D10114968C910E94840883EA95E0BF
:106AE0000E9437178EE298E00E943717C2010E9479
:106AF000370DEAA1FBA1EF2BA1F04B015C012A8D20
:106B00003B8D4C8D5D8D821A930AA40AB50AB7FE9F
:106B100008C0B094A09490948094811C911CA11CF6
:106B2000B11C4B815C81452B19F58DE795E00E94E6
:106B3000371782E596E00E94371784ED93E00E94B4
:106B4000371788A199A10E94321782E596E00E942A
:106B500037178FE598E00E943717C501B4010E94EE
:106B6000115E42E00E94561B0E942A160E94C8191C
:106B700085E090E0AC85BD858D939C9345E050E029
:106B8000B1018AA99BA9ADD9C1010E94A1110E949E
:106B9000B2160E94321BB1E06B16710409F45FCE8D
:106BA000E2E06E16710409F462CE0E942A16DC013E
:106BB0001E968D929D92AD92BC9251970E942A167C
:106BC0000E94D11CEC85FD851182108250E040E0CE
:106BD000B1018AA99BA985D970E060E0C1010E943A
:106BE000D8190E942A16EB81FC81DC019796FC9350
:106BF000EE9396973F01AECAFA01DB01A158BF4F51
:106C00002C91222331F122E030E0DB01AF57BF4F5E
:106C10004C91442311F023E030E0DB01A058BF4F3A
:106C20004C91442311F024E030E0DB01AE57BF4F1C
:106C30004C91442311F026E030E04081518142170D
:106C4000530761F0121613063CF431832083A90127
:106C500048C930E020E0D9CF1182108208952F92E8
:106C60003F924F925F926F927F928F929F92AF92DC
:106C7000BF92CF92DF92EF92FF920F931F93CF9329
:106C8000DF93CDB7DEB7C255D1090FB6F894DEBF9A
:106C90000FBECDBF1C012A013B01098B1A8B2B8B28
:106CA0003C8BAA960EAD1FADAA97FC01E151FD4F9A
:106CB00060817181828193810E94115EA3019201A2
:106CC0000E94705E0E9467606D877E878F87988BB9
:106CD000F101ED50FD4F60817181828193810E94AD
:106CE000115E29893A894B895C890E94705E0E94F5
:106CF0006760698F7A8F8B8F9C8FF101E950FD4F10
:106D000060817181828193810E94115EA701960149
:106D10000E94705E0E94676069A77AA78BA79CA7F4
:106D20000E94250A2B013C01F101E459FD4F11821B
:106D300010823296118210827296A114B10461F011
:106D4000C501B0E0A0E04081518162817381841768
:106D50009507A607B70714F0A080B180F101EC57A2
:106D6000FD4F80819181A281B3818114910441F012
:106D7000A40170E060E0481759076A077B070CF030
:106D80004C01F101E857FD4F80819181A281B381CF
:106D90000115110541F0A80170E060E0481759079E
:106DA0006A077B070CF08C019101205F3F4F3E8BFF
:106DB0002D8BC501B0E0A0E0F10184AF95AFA6AF87
:106DC000B7AF2A563F4F3A8B298BB12CA12CD90152
:106DD0009C968D929D92AD92BC929F974101B4EC8E
:106DE0008B1ABEEF9B0A30E020E0F40104A715A740
:106DF00026A737A70E942A160E942A160E942A1642
:106E00000E942A16DC011E962D913D914D915C91B8
:106E100051972F8F38A349A35AA30E942A16DC0149
:106E200052962D913D914D915C9155972DA33EA386
:106E30004FA358A70E942A16DC0156962D913D912A
:106E40004D915C9159972F83388749875A87F10173
:106E5000E550FD4F10821182128213823496108207
:106E6000118212821382349610821182128213824E
:106E700034961182108232961182108232961182DB
:106E8000108232962F8D38A149A15AA120833183D7
:106E90004283538334968DA19EA1AFA1B8A5808370
:106EA0009183A283B38334962F81388549855A858F
:106EB0002083318342835383AB96EFACAB970D8530
:106EC0001E852F8538894F8D58A169A17AA18D899A
:106ED0009E890E94FA118823F9F082E592E00E94CF
:106EE00037178FE494E00E943717F101EA59FF4FFA
:106EF0006081718182819381E757FD4F20813181CB
:106F0000428153810E943D5FCA01B9010E940A1764
:106F10000E942A160E94C819AC96EFACAC97098D56
:106F20001A8D2B8D3C8D4DA15EA16FA178A589890D
:106F30009A890E94FA118823F9F08EE492E00E9467
:106F400037178FE594E00E943717F101E450FF4FA7
:106F50006081718182819381E950FE4F208131816E
:106F6000428153810E943D5FCA01B9010E940A1704
:106F70000E942A160E94C819AD96EFACAD9709A5DC
:106F80001AA52BA53CA54F81588569857A85C40132
:106F90000E94FA118823F9F08AE492E00E943717E0
:106FA0008FE694E00E943717F101EE56FE4F6081A4
:106FB000718182819381EB59FE4F20813181428121
:106FC00053810E943D5FCA01B9010E940A170E94C5
:106FD0002A160E94C819D10155961C92F101E55557
:106FE000FF4F1082EA56FF4F10820E94B2160E9495
:106FF000321B8D899E890E94C11389899A890E94BA
:10700000C113C4010E94C11381E090E0F101E9586D
:10701000FD4F918380837101B7E8EB1ABDEFFB0A46
:10702000F70191838083810105581D4FD8018D930D
:107030009C9341E050E06D897E89C1010E94712FCF
:10704000F7014081518169897A89C1010E94712FBC
:10705000D8014D915C91B401C1010E94712F11E0E2
:10706000F101E45AFC4F10838D899E890E94E21140
:1070700089899A890E94E211C4010E94E21164E6A2
:1070800070E080E090E00E94F409D101AC58BD4F5F
:107090001C9391012B583D4FF9011083C1018A586F
:1070A0009D4FFC011083AB96FFADAB97F1110FC064
:1070B000AC964FADAC97411105C0AD965FADAD97A5
:1070C000552349F1C10185579F4FFC011082AC96B1
:1070D000FFADAC97F11105C0C1018F5D9E4FFC0162
:1070E0001082AD96FFADAD97F11105C0C101895475
:1070F0009E4FFC011082AB96FFADAB97FC93AC9614
:10710000EFADAC97D901EC93F101EA58FD4FAD9684
:107110002FADAD972083F101E957FF4F1082118207
:1071200012821382EA56FF4F10821182128213825A
:10713000EA56FF4F10821182128213828D899E8936
:107140000E94401789899A890E944017C4010E94B1
:1071500040178D899E890E94031389899A890E940C
:107160000313C4010E9403130E942A16DC01D49663
:107170008C918D871BAA1CAA1DAA1EAA1FAA18AE35
:1071800019AE1AAE1BAE1CAE1DAE1EAEB12CA12C9C
:10719000F101EC58FD4FFA8FE98F91012B583D4FCB
:1071A0003AA729A7A1014A585D4F5EA74DA7C10183
:1071B00089589D4F23969FAF8EAF2397D101A75833
:1071C000BD4F2596BFAFAEAF259737962796FFAF39
:1071D000EEAF2797275E314021963FAF2EAF219724
:1071E0004F535F4F29965FAF4EAF299706962B9668
:1071F0009FAF8EAF2B97AE54BF4F2D96BFAFAEAFA4
:107200002D97EF52FF4F2F96FFAFEEAF2F972557D9
:107210003D4F61963FAF2EAF61974A525109639639
:107220005FAF4EAF6397A98DBA8D8C9181110AC063
:10723000E9A5FAA58081811105C0ADA5BEA58C91F7
:10724000882319F0BD85BB2369F081010A591D4FC0
:10725000D8018D919C91892B09F4EBC5C1010E9445
:107260007E2EF6CFC1010E94E11023964EAD5FAD98
:1072700023976D897E89C101BFDC25964EAD5FAD38
:10728000259769897A89C101B7DC27964EAD5FAD34
:107290002797B401C101B0DC8D899E890E946E13CD
:1072A00089899A890E946E13C4010E946E132196E7
:1072B000EEADFFAD21978081882309F452C08D89FE
:1072C0009E890E9440172996AEADBFAD29978C913B
:1072D0008823D1F02D96CEACDFAC2D972F96EEAC57
:1072E000FFAC2F9761960EAD1FAD619763962EADE3
:1072F0003FAD6397A10145505D4FB1016E527E4F86
:107300008D899E890E942D102196EEADFFAD2197AB
:107310001082AB96FFADAB97FF2319F12B96AEAD64
:10732000BFAD2B978C91811116C02F8D38A149A12B
:107330005AA112161306140615069CF02BAD3CAD8F
:107340004DAD5EAD2F5F3F4F4F4F5F4F2BAF3CAF0B
:107350004DAF5EAF06C08F8D98A1A9A1BAA1B7FFAE
:10736000EDCFF101EC5DFE4F8081882309F44DC023
:1073700089899A890E944017F101E85CFC4F80815D
:107380008823D1F0610131EDC31A3CEFD30A7101BA
:1073900042EBE41A4CEFF40A8101035E1C4F9101A9
:1073A0002F5E3C4FA10141505D4FB1016E5F7D4F9B
:1073B00089899A890E942D10F101EC5DFE4F10829F
:1073C000AC965FADAC97552301F1E65AFE4F808134
:1073D000811115C08DA19EA1AFA1B8A518161906DF
:1073E0001A061B0694F08FA998ADA9ADBAAD019607
:1073F000A11DB11D8FAB98AFA9AFBAAF06C02DA12B
:107400003EA14FA158A557FFEECFF101E654FE4F24
:107410008081882309F44CC0C4010E944017F10107
:10742000E75CFC4F80818823C9F061019DECC91A9B
:107430009CEFD90A7101A0EBEA1AACEFFA0A8101BC
:107440000F5D1C4F91012B5E3C4FA1014D5F5C4FC6
:10745000B1016E5C7D4FC4010E942D10F101E65414
:10746000FE4F1082AD96BFADAD97BB2309F1EB5334
:10747000FF4F8081811116C02F81388549855A853B
:1074800012161306140615069CF02BA93CA94DA94B
:107490005EA92F5F3F4F4F4F5F4F2BAB3CAB4DABC8
:1074A0005EAB06C08F819885A985BA85B7FFEDCF01
:1074B000810105571F4FD8018C91882309F442C0E0
:1074C000F101EB5DFC4F60817181072E000C880B90
:1074D000990B0E94115E9B01AC01F101E550FD4F3B
:1074E00060817181828193810E94986087FD2AC0AA
:1074F000F801108268E973E009521E4FC8010E942A
:10750000402F61EB75E0C8010E94402F6DEC75E0E3
:10751000C8010E94402F6EE278E0C8010E94402F0F
:10752000AB96FFADAB97FF2309F45DC1C1018E524D
:107530009E4F0E94CD0FF101EE59FF4F1082118234
:107540001282138281010F5D1E4FD8018C91882316
:1075500009F442C0F101E95DFC4F60817181072EA1
:10756000000C880B990B0E94115E9B01AC01F1018C
:10757000E150FD4F60817181828193810E9498600A
:1075800087FD2AC0F801108268E973E00F5B1E4F87
:10759000C8010E94402F6AED75E0C8010E94402F8B
:1075A0006DEC75E0C8010E94402F6EE278E0C801E2
:1075B0000E94402FAC96FFADAC97FF2309F417C192
:1075C000C1018E5F9D4F0E94CD0FF101E850FF4F2A
:1075D0001082118212821382810109541E4FD80138
:1075E0008C91882309F442C0F101E75DFC4F608172
:1075F0007181072E000C880B990B0E94115E9B0174
:10760000AC01F101ED5FFC4F60817181828193815A
:107610000E94986087FD2AC0F801108268E973E033
:1076200005551F4FC8010E94402F66EF75E0C80145
:107630000E94402F6DEC75E0C8010E94402F6EE261
:1076400078E0C8010E94402FAD96FFADAD97FF23B3
:1076500009F4D1C0C1018E5C9D4F0E94CD0FF10194
:10766000E257FE4F108211821282138260E08D89F0
:107670009E890E947C12882361F0F101EE59FF4F30
:107680001082118212821382C1018E529E4F0E947B
:10769000CD0F60E089899A890E947C12882361F06D
:1076A000F101E850FF4F1082118212821382C10152
:1076B0008E5F9D4F0E94CD0F60E0C4010E947C123E
:1076C000882361F0F101E257FE4F1082118212828D
:1076D0001382C1018E5C9D4F0E94CD0FF101E557D1
:1076E000FF4F8081A98DBA8D8C93EA56FF4F808120
:1076F000E9A5FAA58083F101E954FE4F8081ADA58B
:10770000BEA58C93E555F1402081318142815381A2
:107710002F8F38A349A35AA3EA56FF4F8081918146
:10772000A281B3818DA39EA3AFA3B8A7EA56FF4F52
:1077300020813181428153812F83388749875A873D
:107740000E942A162F8D38A149A15AA1DC011E964C
:107750002D933D934D935C9351970E942A162DA132
:107760003EA14FA158A5DC0152962D933D934D9318
:107770005C9355970E942A162F81388549855A8532
:10778000DC0156962D933D934D935C9359970E943F
:10779000B216E98DFA8D8081882309F45EC00E94BB
:1077A000250A641575058605970548F50E94250A82
:1077B000641575058605970508F04FC00E94250AD7
:1077C0006B017C01F101ED51FD4F2081318142813E
:1077D0005381A8EEB3E00E94595F6C157D058E05BC
:1077E0009F0530F13AC07FE1A72EB12CABCE60E20D
:1077F000A62EB12CF1CE51E2A52EB12C37CF0E948E
:10780000250A6B017C01C418D508E608F708F101C8
:10781000ED51FD4F2081318142815381A8EEB3E0CB
:107820000E94595F6C157D058E059F0508F0BECF3F
:1078300066E672E081010E591D4FC8010E94402F7B
:107840006EE278E0C8010E94402F62E075E0C80156
:107850000E94402F42E0A42EB12CA9A5BAA58C917C
:10786000882309F451C00E94250A64157505860510
:107870009705E8F40E94250A6415750586059705A5
:1078800008F042C00E94250A6B017C01F101E95118
:10789000FD4F2081318142815381A8EEB3E00E94E7
:1078A000595F6C157D058E059F05C8F02DC00E949F
:1078B000250A6B017C01C418D508E608F708F10118
:1078C000E951FD4F2081318142815381A8EEB3E01F
:1078D0000E94595F6C157D058E059F0558F662E67E
:1078E00072E081010E591D4FC8010E94402F6EE2C7
:1078F00078E0C8010E94402F67E175E0C8010E944E
:10790000402F32E0A32EB12CEDA5FEA58081882367
:1079100009F451C00E94250A64157505860597056E
:10792000E8F40E94250A641575058605970508F098
:1079300042C00E94250A6B017C01F101E551FD4F17
:107940002081318142815381A8EEB3E00E94595FCA
:107950006C157D058E059F05C8F02DC00E94250A77
:107960006B017C01C418D508E608F708F101E55160
:10797000FD4F2081318142815381A8EEB3E00E9406
:10798000595F6C157D058E059F0558F66EE572E012
:1079900081010E591D4FC8010E94402F6EE278E010
:1079A000C8010E94402F6CE275E0C8010E94402F80
:1079B00022E0A22EB12C8CE09DE00E940108181656
:1079C00019060CF040C08CE09DE00E94DF078F7D1F
:1079D00085349105C1F561E475E0C1018E599D4F73
:1079E0000E94402F8AE592E00E9437170E942A16D3
:1079F0000E94C819F101E557FF4F1082EA56FF4F68
:107A00001082EA56FF4F1082A98DBA8D1C92E9A50B
:107A1000FAA51082ADA5BEA51C92B1E0BD87AA242F
:107A2000A394B12C62E176E0C1018E599D4F0E9472
:107A3000402FE98DFA8D1082A9A5BAA51C92EDA55B
:107A4000FEA5108203C0A114B10461F7C1010E9418
:107A50007E2EF101E259FD4F808191810196918343
:107A600080838D3291400CF4DECBD101AA59BD4FF9
:107A70008D919C911197892B09F0D5CB14968D91FE
:107A80009C91892B09F0CFCB118210823297808193
:107A900091810097A1F0019761F1F101E459FD4F47
:107AA000808191810196823091050CF0BFC1918354
:107AB0008083F101E659FD4F11821082B4CB66E557
:107AC00072E081010E591D4FC8010E94402F0E9493
:107AD0002A16BC01CE0101960E94492FBE016F5F9C
:107AE0007F4FC8010E946B2FCE0101960E94661D38
:107AF000D4CF0E942A168C01FC0180819181A28141
:107B0000B381181619061A061B0644F081E090E0AE
:107B1000A0E0B0E080839183A283B383F8018481E5
:107B20009581A681B781181619061A061B0644F01E
:107B300081E090E0A0E0B0E084839583A683B783E2
:107B4000F80180859185A285B385181619061A0655
:107B50001B0644F081E090E0A0E0B0E080879187D0
:107B6000A287B3871A8219821C821B821E821D8201
:107B7000CE0101960E949E2B6AE374E0CE0101962D
:107B80000E94402F6FE474E0CE0101960E94402FC6
:107B9000D8011E966D917D918D919C9151970E9477
:107BA000115E6B017C01F80160817181828193819A
:107BB0000E94115E9B01AC01C701B6010E94FF5FEC
:107BC000AB01BC01CE0101960E94E02E6FE574E08E
:107BD000CE0101960E94402FD80152966D917D9161
:107BE0008D919C9155970E94115E6B017C01F8016B
:107BF00064817581868197810E94115E9B01AC0131
:107C0000C701B6010E94FF5FAB01BC01CE01019626
:107C10000E94E02E6FE674E0CE0101960E94402F94
:107C2000D80156966D917D918D919C9159970E94A6
:107C3000115E6B017C01F8016085718582859385F9
:107C40000E94115E9B01AC01C701B6010E94FF5F5B
:107C5000AB01BC01CE0101960E94E02EBE016F5F18
:107C60007F4F81010E591D4FC8010E946B2FCE011D
:107C700001960E94661D0E942A16BC01CE01019643
:107C80000E94492FBE016F5F7F4FC8010E946B2F7A
:107C9000CE0101960E94661D6AE372E0C8010E944F
:107CA000402F6FE474E0C8010E94402F91012E52D2
:107CB0003E4F3C872B87C9010E94370D0E94115E01
:107CC0006B017C01F101E151FD4F60817181828185
:107CD00093810E94115E9B01AC01C701B6010E9415
:107CE000FF5FAB01BC01C8010E94E02E6FE574E0AC
:107CF000C8010E94402FA1014E5F5D4F5CA34BA3C2
:107D0000CA010E94370D0E94115E6B017C01F101D6
:107D1000ED50FD4F60817181828193810E94115EDF
:107D20009B01AC01C701B6010E94FF5FAB01BC0122
:107D3000C8010E94E02E6FE674E0C8010E94402F47
:107D400071015EECE51A5DEFF50AC7010E94370D7F
:107D50000E94115E6FA778AB89AB9AABF101E95035
:107D6000FD4F60817181828193810E94115E9B0130
:107D7000AC016FA578A989A99AA90E94FF5FAB0100
:107D8000BC01C8010E94E02E0E942A16BC01CE014F
:107D900001960E94492FBE016F5F7F4FC8010E946C
:107DA0006B2FCE0101960E94661D66E372E0C8014A
:107DB0000E94402F6FE474E0C8010E94402FEB85C1
:107DC000FC85A68DB78D20893189428953890E940F
:107DD000635FAB01BC01C8010E94102F6FE574E026
:107DE000C8010E94402FEBA1FCA1A68DB78D208970
:107DF0003189428953890E94635FAB01BC01C8018C
:107E00000E94102F6FE674E0C8010E94402FF70116
:107E1000A68DB78D20893189428953890E94635F7D
:107E2000AB01BC01C8010E94102F51CE11821082FB
:107E300040CE8EE196E00E943717AB96BFADAB9770
:107E4000BB2379F1A114B104B9F5ED85E11134C07A
:107E500086E492E00E9437170E942A160E94C819F1
:107E6000AC96FFADAC97FF2341F082E492E00E9414
:107E700037170E942A160E94C819AD964FADAD97CC
:107E80004423D1F0A114B104B9F45D85511114C09B
:107E90008EE392E00E9437170E942A160E94C819AA
:107EA0000BC0AC963FADAC97332339F3A114B104AA
:107EB00019F42D852223C9F2C10189589D4F9E8F47
:107EC0008D8F85E090E0AD8DBE8D8D939C9381016B
:107ED00007581D4FF80191838083910125583D4F2C
:107EE000388F2F8BD9018D939C9345E050E06D899D
:107EF0007E89C1010E94712FF801408151816989F9
:107F00007A89C1010E94712FAF89B88D4D915C9122
:107F1000B401C1010E94712FC1010E94B811F10189
:107F2000EE59FF4F4080518062807380EA56FF4FC8
:107F300020813181428153812F83388749875A8735
:107F4000EA56FF4FC080D180E280F3800E942A165B
:107F5000DC011E964D925D926D927C9251970E942B
:107F60002A162F81388549855A85DC0152962D9332
:107F70003D934D935C9355970E942A16FC01C68A47
:107F8000D78AE08EF18E0E942A162BAD3CAD4DAD06
:107F90005EADDC0198962D933D934D935C939B973A
:107FA0000E942A162FA938AD49AD5AADDC019C9626
:107FB0002D933D934D935C939F970E942A162BA976
:107FC0003CA94DA95EA9DC01D0962D933D934D931C
:107FD0005C93D3970E94B2160E94321B0E942A160D
:107FE0000E94D11CC1010E942B1CED8DFE8D1182BF
:107FF0001082D8011D921C92EF89F88D1182108297
:1080000050E040E06D897E89C1010E94712FD80146
:108010004D915C9169897A89C1010E94712FEF8924
:10802000F88D40815181B401C1010E94712FC101BD
:108030000E94B811FD85FF2349F00E942A1621E015
:10804000DC01D4962C93AA24A394B12C8CE296E064
:108050000E943717C5010E9432178EE298E00E94F5
:1080600037170E942A16FC01B7A2A6A2C501CE5A54
:10807000DF4F0FB6F894DEBF0FBECDBFDF91CF91BB
:108080001F910F91FF90EF90DF90CF90BF90AF9036
:108090009F908F907F906F905F904F903F902F9028
:1080A00008954F925F926F927F928F929F92AF92BC
:1080B000BF92CF92DF92EF92FF920F931F93CF93D5
:1080C000DF9300D01F92CDB7DEB70E94691EC0902B
:1080D000630AD090640AE090650AF090660A0E94F4
:1080E000691E8090670A9090680AA090690AB09013
:1080F0006A0A0E942A16FC014684578460887188A7
:108100000E942A169A838983C301B2010E94115EDC
:108110002B013C01C701B6010E94115E9B01AC011D
:10812000C301B2010E94FF5F2B013C01E981FA818A
:1081300062897389848995890E94115E6B017C0133
:10814000C501B4010E94115E9B01AC01C701B601DB
:108150000E94FF5F69837A838B839C830E94DB2D5F
:108160001F921F921F921F921F92912C812CB12C53
:10817000A12CC12CD12C760109811A812B813C8143
:10818000B301A2010E942F360E94DB2D1F921F9285
:108190001F921F921F9297018601B301A2010E94B4
:1081A0002F360E94DB2D1F921F921F921F921F924B
:1081B0009701B701A6010E942F360FB6F894DEBFD3
:1081C0000FBECDBF90E080E00F900F900F900F900A
:1081D000DF91CF911F910F91FF90EF90DF90CF90A3
:1081E000BF90AF909F908F907F906F905F904F90D7
:1081F00008958F929F92AF92BF92CF92DF92EF92AB
:10820000FF920F931F93CF93DF93EB010E94DB2D1F
:108210008A889B88AE84BF84CA84DB84EC84FD8416
:108220000E811F81288539854A815B816C817D8122
:108230001F921F921F92EF89EF93EE89EF930E9496
:108240002F360F900F900F900F900F9090E080E0DE
:10825000DF91CF911F910F91FF90EF90DF90CF9022
:10826000BF90AF909F908F9008958F929F92AF9202
:10827000BF92CF92DF92EF92FF920F931F930E94D3
:10828000DB2D62E070E00E94C12F892BD1F40E94A7
:10829000DB2D21E02F931F921F921F921F92912C92
:1082A000812CB12CA12CC12CD12C760197018601F7
:1082B000B701A6010E942F360F900F900F900F90DC
:1082C0000F9090E080E01F910F91FF90EF90DF9072
:1082D000CF90BF90AF909F908F9008958F929F9274
:1082E000AF92BF92CF92DF92EF92FF920F931F93C4
:1082F0000E94DB2D61E070E00E94C12F892BD1F438
:108300000E94DB2D1F9221E02F931F921F921F923C
:10831000912C812CB12CA12CC12CD12C7601970150
:108320008601B701A6010E942F360F900F900F9083
:108330000F900F9090E080E01F910F91FF90EF90D1
:10834000DF90CF90BF90AF909F908F9008958F92C5
:108350009F92AF92BF92CF92DF92EF92FF920F93D4
:108360001F930E94DB2D70E060E00E94C12F892BDB
:10837000D1F40E94DB2D1F921F9221E02F931F92B8
:108380001F92912C812CB12CA12CC12CD12C7601C7
:1083900097018601B701A6010E942F360F900F901A
:1083A0000F900F900F9090E080E01F910F91FF9041
:1083B000EF90DF90CF90BF90AF909F908F900895F7
:1083C0002F923F924F925F926F927F928F929F92E5
:1083D000AF92BF92CF92DF92EF92FF920F931F93D3
:1083E000CF93DF93CDB7DEB72F970FB6F894DEBFEC
:1083F0000FBECDBF0E94DB2D21E02F931F921F9255
:108400001F921F92912C812CB12CA12CC12CD12C0C
:10841000760197018601B701A6010E942F360E94BE
:10842000691EE0905B0AF0905C0A0E94691E6090F1
:108430006B0A70906C0A0E94691E80914B0B9091A0
:108440004C0BA0914D0BB0914E0B0F900F900F90D5
:108450000F900F90161417040CF070C19A8789873B
:10846000EA94EF2809F070C186EF9FEF9A83898321
:108470000E942A16FC0166857785808991890E9471
:10848000115E6B017C010E94691E6091630A70910C
:10849000640A8091650A9091660A0E94115E9B01B0
:1084A000AC01C701B6010E94FF5F6D837E838F839D
:1084B00098870E942A16DC0152966D917D918D91CC
:1084C0009C9155970E94115E6B017C010E94691E70
:1084D0006091670A7091680A8091690A90916A0AAE
:1084E0000E94115E9B01AC01C701B6010E94FF5FB3
:1084F0001B012C010E942A160E94691E0E94DB2D7E
:108500001F921F921F921F921F92912C812CB12CAF
:10851000A12CC12CD12C7601920181014D815E816B
:108520006F8178850E942F360E942A16FC0184A94B
:108530008D8789859A85880F991F29853A85280F07
:10854000391F3C872B870F900F900F900F900F9043
:108550001F861E8689819A81092E000CAA0BBB0BEF
:1085600089839A83AB83BC830E94DB2D9A8789879A
:1085700069817A818B819C810E94115E6B017C01F3
:108580001F921F921F921F921F92912C812CB12C2F
:10859000A12C920181014D815E816F817885898551
:1085A0009A850E942F360E942A160F900F900F90E6
:1085B0000F900F90DC01D4968C918111D6C00E944F
:1085C000DB2DB1E0BF931F921F921F921F92C12C0F
:1085D000D12C760192014D815E816F8178850E9458
:1085E0002F360E942A160F900F900F900F900F9029
:1085F000FC0184A98111B9C087E396E00E94371776
:108600008CE496E00E9437170E942A16DC019896A7
:108610006D917D918D919C919B970E940A1780E5A9
:1086200096E00E9437170E942A16FC0160A571A5EA
:1086300082A593A520813181428153810E943D5FB3
:10864000CA01B9010E940A1784E596E00E94371713
:108650000E942A16FC0164A575A586A597A50E940F
:108660000A1780E596E00E9437170E942A16FC013F
:1086700064A575A586A597A5248135814681578176
:108680000E943D5FCA01B9010E940A1788E596E081
:108690000E9437170E942A16DC01D0966D917D91B9
:1086A0008D919C91D3970E940A1780E596E00E94D5
:1086B00037170E942A16FC0160A971A982A993A903
:1086C00020853185428553850E943D5FCA01B901ED
:1086D0000E940A178EE298E00E9437170E942A161D
:1086E000FC018B859C85B3010E94BB606B01B4E1EA
:1086F000CB0ED11C0D2C000CEE08FF0860A971A94F
:1087000082A993A920853185428553850E943D5FCA
:108710002C153D054E055F05E4F4EE85FF85319689
:10872000FF87EE873397ECF00E942A16DC015696FD
:108730001D921D921D921C92599717C01A86198678
:1087400066246394712C8CCEAAE0B0E0BA83A9832E
:108750008FCE64EF71E080E090E00E94F4091F8604
:108760001E869D85992309F4FFCE90E080E02F9628
:108770000FB6F894DEBF0FBECDBFDF91CF911F9132
:108780000F91FF90EF90DF90CF90BF90AF909F90B0
:108790008F907F906F905F904F903F902F900895B3
:1087A0002F923F924F925F926F927F928F929F9201
:1087B000AF92BF92CF92DF92EF92FF920F931F93EF
:1087C000CF93DF93CDB7DEB761970FB6F894DEBFD6
:1087D0000FBECDBF0E94691E2091570A3091580AE2
:1087E0003E832D830E94691E8091670A9091680ADA
:1087F0009A8389830E94691E8091470B9091480B50
:10880000A091490BB0914A0BE981FA811E161F060F
:108810000CF057C19C838B838D819E81019709F059
:1088200057C1A6EFBFEFBD87AC870E942A16DC01B7
:108830001E966D917D918D919C9151970E94115E34
:108840006B017C010E94691E6091630A7091640A49
:108850008091650A9091660A0E94115E9B01AC01AD
:10886000C701B6010E94FF5F6D837E838F83988767
:108870000E942A160E94691E0E942A16FC0166891F
:108880007789808D918D0E94115E6B017C010E9421
:10889000691E60916B0A70916C0A80916D0A9091CB
:1088A0006E0A0E94115E9B01AC01C701B6010E94D5
:1088B000FF5F2B013C010E94DB2D1F921F921F9234
:1088C0001F921F92912C812CB12CA12C730162015B
:1088D00000E010E098014D815E816F8178850E94F3
:1088E0002F360E942A16DC01D4968C918B878B81BF
:1088F0009C81880F991FEB81FC81E80FF91FFA8793
:10890000E9870F900F900F900F900F90312C212C32
:108910008C859D85092E000CAA0BBB0B8C879D872F
:10892000AE87BF870E94DB2D998B888B6C857D85F8
:108930008E859F850E94115E8B019C011F921F9264
:108940001F921F921F92912C812CB12CA12C73018C
:1089500062014D815E816F817885888999890E9445
:108960002F360E942A160F900F900F900F900F90A5
:10897000DC01D4968C918111BCC00E94DB2D1F922A
:10898000B1E0BF931F921F921F9200E010E0980188
:108990004D815E816F8178850E942F360E942A1654
:1089A0000F900F900F900F900F90FC0184A98111F0
:1089B000A0C087E396E00E9437178CE496E00E94FF
:1089C00037170E942A16FC0160A571A582A593A500
:1089D00020813181428153810E943D5FCA01B901EA
:1089E0000E940A1784E596E00E9437170E942A1613
:1089F000FC0164A575A586A597A5248135814681CE
:108A000057810E943D5FCA01B9010E940A1788E59B
:108A100096E00E9437170E942A16FC0160A971A9EE
:108A200082A993A920853185428553850E943D5FA7
:108A3000CA01B9010E940A178CE596E00E94371717
:108A40008B819C810E9432178CE596E00E9437173B
:108A500089819A810E9432178EE298E00E9437172E
:108A60000E942A16FC0189859A8569817A810E9473
:108A7000BB606B0124E1C20ED11C0D2C000CEE0872
:108A8000FF0864A575A586A597A524813581468133
:108A900057810E943D5FC216D306E406F506ECF04E
:108AA0003FEF231A330A83E028163104F4F00E94C2
:108AB0002A16DC0152961D921D921D921C9255970A
:108AC00018C01C821B8221E030E03A832983A4CEA7
:108AD000EAE0F0E0FD87EC87A8CE64EF71E080E08B
:108AE00090E00E94F409312C212C9B85992309F4F4
:108AF00019CF90E080E061960FB6F894DEBF0FBE0C
:108B0000CDBFDF91CF911F910F91FF90EF90DF903C
:108B1000CF90BF90AF909F908F907F906F905F901D
:108B20004F903F902F9008952F923F924F925F92D7
:108B30006F927F928F929F92AF92BF92CF92DF926D
:108B4000EF92FF920F931F93CF93DF93CDB7DEB7D2
:108B50002F970FB6F894DEBF0FBECDBF0E94691EDF
:108B6000E090530AF090540A0E94691E6090630AD4
:108B70007090640A0E94691E8091430B9091440B8F
:108B8000A091450BB091460B161417040CF06FC161
:108B90009A878987EA94EF2809F06FC186EF9FEFE3
:108BA0009A8389830E942A160E94691E0E942A16AF
:108BB000FC0162897389848995890E94115E6B0129
:108BC0007C010E94691E6091670A7091680A809119
:108BD000690A90916A0A0E94115E9B01AC01C7016B
:108BE000B6010E94FF5F6D837E838F8398870E940A
:108BF0002A16DC0156966D917D918D919C91599725
:108C00000E94115E6B017C010E94691E60916B0ADB
:108C100070916C0A80916D0A90916E0A0E94115EAB
:108C20009B01AC01C701B6010E94FF5F1B012C0133
:108C30000E94DB2D1F921F921F921F921F92912C58
:108C4000812CB12CA12C720161010D811E812F811B
:108C5000388540E050E0BA010E942F360E942A1663
:108C6000FC0184A98D8789859A85880F991F29859C
:108C70003A85280F391F3C872B870F900F900F9054
:108C80000F900F901F861E8689819A81092E000CF5
:108C9000AA0BBB0B89839A83AB83BC830E94DB2D19
:108CA0009A87898769817A818B819C810E94115E74
:108CB000AB01BC011F921F921F921F921F92912C19
:108CC000812CB12CA12C720161010D811E812F819B
:108CD000388589859A850E942F360E942A160F9022
:108CE0000F900F900F900F90DC01D4968C91811112
:108CF000D5C00E94DB2D1F921F92B1E0BF931F923F
:108D00001F920D811E812F81388540E050E0BA010D
:108D10000E942F360E942A160F900F900F900F90EE
:108D20000F90FC0184A98111B9C087E396E00E94ED
:108D300037178CE496E00E9437170E942A16DC0150
:108D400098966D917D918D919C919B970E940A17A9
:108D500080E596E00E9437170E942A16FC0160A564
:108D600071A582A593A520813181428153810E9402
:108D70003D5FCA01B9010E940A1784E596E00E948E
:108D800037170E942A16FC0164A575A586A597A52C
:108D90000E940A1780E596E00E9437170E942A1663
:108DA000FC0164A575A586A597A52481358146811A
:108DB00057810E943D5FCA01B9010E940A1788E5E8
:108DC00096E00E9437170E942A16DC01D0966D911A
:108DD0007D918D919C91D3970E940A1780E596E032
:108DE0000E9437170E942A16FC0160A971A982A966
:108DF00093A920853185428553850E943D5FCA0134
:108E0000B9010E940A178EE298E00E9437170E946B
:108E10002A16FC018B859C85B3010E94BB606B0107
:108E2000B4E1CB0ED11C0D2C000CEE08FF0860A5A0
:108E300071A582A593A520813181428153810E9431
:108E40003D5F2C153D054E055F05E4F4EE85FF857D
:108E50003196FF87EE873397ECF00E942A16DC01EB
:108E60001E961D921D921D921C92519717C01A8634
:108E7000198666246394712C8DCEAAE0B0E0BA8383
:108E8000A98390CE64EF71E080E090E00E94F40945
:108E90001F861E869D85992309F400CF90E080E00F
:108EA0002F960FB6F894DEBF0FBECDBFDF91CF91E6
:108EB0001F910F91FF90EF90DF90CF90BF90AF90F8
:108EC0009F908F907F906F905F904F903F902F90EA
:108ED00008951F920F920FB60F9211240BB60F92A6
:108EE0002F933F934F935F936F937F938F939F93B2
:108EF000AF93BF93EF93FF938CE09DE00E94160821
:108F0000FF91EF91BF91AF919F918F917F916F9161
:108F10005F914F913F912F910F900BBE0F900FBE1D
:108F20000F901F9018951F920F920FB60F92112459
:108F30000BB60F922F938F939F93EF93FF93E09134
:108F40001C0DF0911D0D8081E091220DF091230DFB
:108F500082FD1DC090818091250D8F5F8F732091C0
:108F6000260D821741F0E091250DF0E0E45FF24F0D
:108F7000958F8093250DFF91EF919F918F912F9168
:108F80000F900BBE0F900FBE0F901F901895808111
:108F9000F2CF1F920F920FB60F9211242F933F938F
:108FA0008F939F93AF93BF938091750890917608AC
:108FB000A0917708B09178083091740823E0230FCE
:108FC0002D3758F50196A11DB11D2093740880938B
:108FD000750890937608A0937708B09378088091ED
:108FE000790890917A08A0917B08B0917C0801964D
:108FF000A11DB11D8093790890937A08A0937B08F6
:10900000B0937C08BF91AF919F918F913F912F9129
:109010000F900FBE0F901F90189526E8230F029611
:10902000A11DB11DD2CF1F920F920FB60F92112426
:109030000BB60F922F933F934F935F936F937F9352
:109040008F939F93AF93BF93EF93FF9348E251E0C9
:1090500064E271E090E080E00E94340BFF91EF91B8
:10906000BF91AF919F918F917F916F915F914F9140
:109070003F912F910F900BBE0F900FBE0F901F903E
:1090800018951F920F920FB60F9211240BB60F92E4
:109090002F933F934F935F936F937F938F939F9300
:1090A000AF93BF93EF93FF9348EA50E064EA70E018
:1090B00083E090E00E94340BFF91EF91BF91AF915C
:1090C0009F918F917F916F915F914F913F912F91E0
:1090D0000F900BBE0F900FBE0F901F9018951F9210
:1090E0000F920FB60F9211240BB60F922F933F934E
:1090F0004F935F936F937F938F939F93AF93BF93A0
:10910000EF93FF9348E950E064E970E082E090E07B
:109110000E94340BFF91EF91BF91AF919F918F917E
:109120007F916F915F914F913F912F910F900BBE67
:109130000F900FBE0F901F9018951F920F920FB6B1
:109140000F9211240BB60F922F933F934F935F937F
:109150006F937F938F939F93AF93BF93EF93FF93FF
:1091600048E850E064E870E081E090E00E94340B51
:10917000FF91EF91BF91AF919F918F917F916F91EF
:109180005F914F913F912F910F900BBE0F900FBEAB
:109190000F901F9018951F920F920FB60F921124E7
:1091A0000BB60F922F933F934F935F936F937F93E1
:1091B0008F939F93AF93BF93EF93FF93E0917E08BC
:1091C000F0917F081995FF91EF91BF91AF919F9119
:1091D0008F917F916F915F914F913F912F910F9060
:1091E0000BBE0F900FBE0F901F901895FF920F931C
:1091F0001F93CF93DF93EC01F62E8C01065F1F4F78
:109200001B861A861D861C861F861E86C8010E9424
:109210009E2BF886198670E060E0C801DF91CF913F
:109220001F910F91FF900C94792B10920F0D1092BB
:109230000E0D88EE93E0A0E0B0E08093100D9093C7
:10924000110DA093120DB093130D82E893E090934B
:109250000D0D80930C0D85EC90E09093190D80938B
:10926000180D84EC90E090931B0D80931A0D80EC08
:1092700090E090931D0D80931C0D81EC90E09093F5
:109280001F0D80931E0D82EC90E09093210D809332
:10929000200D86EC90E09093230D8093220D109288
:1092A000250D1092260D1092270D1092280D68E1C1
:1092B00088E094E19BDF6CE188E194E197DF67E16E
:1092C00088E294E193DF6DE188E394E18FDF68E168
:1092D00088EC93E18BDF6CE188ED93E187DF67E158
:1092E00088EE93E183DF6DE188EF93E17FDFEAE3CE
:1092F000FEE02FEF48EB5BE08091390E803308F001
:1093000083C191E0980F9093390E808390E0DC0147
:10931000AA0FBB1FA80FB91FA755B24F12965C9397
:109320004E93119733968EE0E634F80729F768E1FB
:1093300088E893E15BDF6CE188E993E157DF67E15F
:1093400088EA93E153DF6DE188EB93E14FDF68E159
:1093500088E493E14BDF6CE188E593E147DF67E167
:1093600088E693E143DF6DE188E793E13FDF68E161
:1093700088E093E13BDF6CE188E193E137DF67E16F
:1093800088E293E133DF6DE188E393E12FDF68E169
:1093900088EC92E12BDF6CE188ED92E127DF67E159
:1093A00088EE92E123DF6DE188EF92E11FDF68E153
:1093B00088E892E11BDF6CE188E992E117DF67E161
:1093C00088EA92E113DF6DE188EB92E10FDF68E15B
:1093D00088E492E10BDF6CE188E592E107DF67E169
:1093E00088E692E103DF6DE188E792E1FFDE68E164
:1093F00088E092E1FBDE6CE188E192E1F7DE67E173
:1094000088E292E1F3DE6DE188E392E1EFDE82E053
:1094100090E00E94925824E933E0FC0131832083DC
:109420009093470E8093460E68E188EC91E1DEDE72
:109430006CE188ED91E1DADE67E188EE91E1D6DE5C
:109440006DE188EF91E1D2DE68E188E891E1CEDE5E
:109450006CE188E991E1CADE67E188EA91E1C6DE64
:109460006DE188EB91E1C2DE68E188E491E1BEDE66
:109470006CE188E591E1BADE67E188E691E1B6DE6C
:109480006DE188E791E1B2DE68E188E091E1AEDE6E
:109490006CE188E191E1AADE67E188E291E1A6DE74
:1094A0006DE188E391E1A2DE68E188EC90E19EDE67
:1094B0006CE188ED90E19ADE67E188EE90E196DE5E
:1094C0006DE188EF90E192DE68E188E890E18EDE60
:1094D0006CE188E990E18ADE67E188EA90E186DE66
:1094E0006DE188EB90E182DE68E188E490E17EDE68
:1094F0006CE188E590E17ADE67E188E690E176DE6E
:109500006DE188E790E172DE68E188E090E16EDE6F
:109510006CE188E190E16ADE67E188E290E166DE75
:109520006DE188E390E162DE68E188EC9FE05EDE59
:109530006CE188ED9FE05ADE67E188EE9FE056DE41
:109540006DE188EF9FE052DE68E188E89FE04EDE43
:109550006CE188E99FE04ADE67E188EA9FE046DE49
:109560006DE188EB9FE042DE68E188E49FE03EDE4B
:109570006CE188E59FE03ADE67E188E69FE036DE51
:109580006DE188E79FE032DE68E188E09FE02EDE53
:109590006CE188E19FE02ADE67E188E29FE026DE59
:1095A0006DE188E39FE022DE68E188EC9EE01EDE4C
:1095B0006CE188ED9EE01ADE67E188EE9EE016DE43
:1095C0006DE188EF9EE012DE68E188E89EE00EDE45
:1095D0006CE188E99EE00ADE67E188EA9EE006DE4B
:1095E0006DE188EB9EE002DE68E188E49EE0FEDD4E
:1095F0006CE188E59EE0FADD67E188E69EE0F6DD55
:109600006DE188E79EE0F2CD20838CCE789484B51E
:10961000826084BD84B5816084BD85B5826085BD6E
:1096200085B5816085BD80916E00816080936E00FC
:1096300010928100809181008260809381008091EE
:10964000810081608093810080918000816080939F
:1096500080008091B10084608093B1008091B0005F
:1096600081608093B000809191008260809391002E
:109670008091910081608093910080919000816041
:10968000809390008091A10082608093A1008091DE
:10969000A10081608093A1008091A00081608093EF
:1096A000A00080912101826080932101809121019D
:1096B000816080932101809120018160809320014D
:1096C00080917A00846080937A0080917A00826031
:1096D00080937A0080917A00816080937A008091F3
:1096E0007A00806880937A001092C100E0911C0D8E
:1096F000F0911D0D82E08083E091180DF091190D1D
:109700001082E0911A0DF0911B0D10E11083109260
:10971000240DE091200DF091210D86E08083E091F1
:109720001E0DF0911F0D808180618083E0911E0DE0
:10973000F0911F0D808188608083E0911E0DF09173
:109740001F0D808180688083E0911E0DF0911F0DB8
:1097500080818F7D808364E670E080E090E00E94ED
:10976000F4098FE692E00E9437178DE692E00E949E
:10977000371780E696E00E9437178AE692E00E944B
:1097800037178FE692E00E9437178DE692E00E942D
:1097900037178AE796E00E9437178AE692E00E9420
:1097A000371761E089E10E94930961E08BE10E9433
:1097B000930961E08AE10E94930962E085E40E94D6
:1097C000930962E084E40E94930961E089E10E94C8
:1097D000660960E08BE10E94660960E08AE10E9410
:1097E000660961E08FE10E94930961E081E20E94D5
:1097F000930961E080E20E94930962E083E40E94A1
:10980000930962E082E40E94930961E08FE10E9483
:10981000660960E081E20E94660960E080E20E94E1
:10982000660961E082E20E94930961E084E20E949D
:10983000930961E083E20E94930962E081E40E945F
:10984000930962E080E40E94930961E082E20E9451
:10985000660960E084E20E94660960E083E20E949B
:10986000660961E08EE00E94930961E08EE10E944A
:10987000930961E08FE00E94930961E08EE00E940D
:10988000660960E08EE10E94660960E08FE00E9458
:10989000660961E088E20E94930961E089E20E9422
:1098A000930961E085E20E94930960E088E20E94EA
:1098B000660960E089E20E94660960E085E20E9434
:1098C000660961E08DE00E94930961E089E00E94F1
:1098D000930961E088E00E94930961E087E00E94BB
:1098E000930961E08AE00E94930961E08CE00E94A4
:1098F000930960E08DE00E94660960E089E00E94C3
:10990000660960E088E00E94660960E087E00E94E6
:10991000660960E08AE00E94660960E08CE00E94CF
:10992000660962E08FE30E94930962E08BE30E9484
:10993000930961E084E00E94930961E085E00E9460
:10994000930961E086E00E94930961E08BE00E9448
:10995000930960E084E00E94660960E085E00E946F
:10996000660960E086E00E94660960E08BE00E9484
:10997000660984EF91E0909303028093020262E013
:1099800081E30E94930961E086E10E94930961E00E
:1099900086E10E9466098CB58F7D8CBD8CB5837F76
:1099A0008CBD0E949C070E94EC0B8FE692E00E9407
:1099B00037178DE692E00E9437178BE996E00E94F8
:1099C00037178AE692E00E9437170E94691E0E94AC
:1099D000E11A8FE692E00E9437178DE692E00E942E
:1099E00037178BEA96E00E9437178AE692E00E94CA
:1099F00037178FE692E00E9437178DE692E00E94BB
:109A000037178CEB96E00E9437178AE692E00E94A7
:109A100037170E94DB2DEC0140960E941014CE01F6
:109A20008A559F4F0E941014CE01845C9E4F0E9465
:109A300010148FE692E00E9437178DE692E00E94A4
:109A4000371781ED96E00E9437178AE692E00E9470
:109A500037170E94DB2DEC010E949E2ACE010E9446
:109A6000732ACE010E94482A8FE692E00E9437179F
:109A70008DE692E00E94371789EE96E00E94371734
:109A80008AE692E00E9437170E94DB2D0E9401298E
:109A90008FE692E00E9437178DE692E00E9437171A
:109AA00080E097E00E9437178AE692E00E9437171D
:109AB00061E089E10E94660961E08EE00E9466092A
:109AC00061E08FE10E94660961E082E20E9466091E
:109AD0008FE692E00E9437178DE692E00E943717DA
:109AE00086E197E00E9437178AE692E00E943717D6
:109AF0000E94571F0E94271F0E94250A0E94250AC4
:109B00006093800870938108809382089093830803
:109B10008FE692E00E9437178DE692E00E94371799
:109B200086E297E00E9437178AE692E00E94371794
:109B300084EF9DE290937F0880937E08C1E0C093FC
:109B40006F001093810010928000C0937D0880E028
:109B500092E0909387008093860081E1809381005A
:109B600010928100109285001092840080917D08EF
:109B70008061809381000E94250A6093830970931D
:109B8000840980938509909386098FE692E00E946C
:109B900037178DE692E00E94371786E397E00E9420
:109BA00037178AE692E00E9437170E94691E80915B
:109BB0008F0990919009A0919109B0919209019714
:109BC000A105B10559F50E94691E8091D7099091B0
:109BD000D809A091D909B091DA090197A105B10579
:109BE000E9F48BE497E00E9437170E94DB2DCF93B6
:109BF0001F921F921F921F92912C812CB12CA12C8D
:109C0000C12CD12C760197018601B701A6010E94D3
:109C10002F360F900F900F900F900F900E94691E9B
:109C200080918F0990919009A0919109B09192092A
:109C30000197A105B10561F50E94691E8091D309C4
:109C40009091D409A091D509B091D6090197A105A9
:109C5000B105F1F483E697E00E9437170E94DB2DEF
:109C60001F9221E02F931F921F921F92912C812C03
:109C7000B12CA12CC12CD12C760197018601B70102
:109C8000A6010E942F360F900F900F900F900F900B
:109C90000E94691E80918F0990919009A09191096D
:109CA000B09192090197A105B10561F50E94691E65
:109CB0008091CF099091D009A091D109B091D2099A
:109CC0000197A105B105F1F48BE797E00E943717E2
:109CD0000E94DB2D1F921F9221E02F931F921F9253
:109CE000912C812CB12CA12CC12CD12C7601970167
:109CF0008601B701A6010E942F360F900F900F909A
:109D00000F900F9088E792E00E94371786E792E065
:109D10000E94371783E997E00E94371783E792E0A4
:109D20000E943717EEE06E2E712CFEEE2F2EF2E021
:109D30003F2E0E94DB2D0E94E1100E94250AAB01FC
:109D4000BC018091800890918108A0918208B09117
:109D50008308481759076A077B0708F060C04093DB
:109D600080085093810860938208709383088CE088
:109D70009DE00E940108892B09F433C30E94250A43
:109D80006093830970938409809385099093860971
:109D90008CE09DE00E94DF0780937909982F9F7DDA
:109DA000953409F468C02091770930917809F90158
:109DB000ED5EF64F80832F5F3F4F309378092093FD
:109DC000770980917709909178098336910564F03D
:109DD0002AE020937909FC01ED5EF64F208301967D
:109DE00090937809809377092091770930917809C9
:109DF000809179098A3021F0243631050CF4F1C2C2
:109E0000C9010197AEEAB8E0E3E1F9E0AF014351DF
:109E1000594048175907B4F541914D93F7CF481B66
:109E2000590B6A0B7B0B483E53406105710508F4E2
:109E30009ECF88519C4FAF4FBF4F80938008909327
:109E40008108A0938208B09383080E94571FEC01F9
:109E50000E94521ACE010C960E94521ACE014896C8
:109E60000E94521ACE0184960E94521ACE01C096C8
:109E70000E94521A7CCF0E942A1621E0DC01D4965F
:109E80002C939FCF8255974FFC01108222303105D1
:109E90000CF4A3C28AE693E00E94371782E596E0AD
:109EA0000E9437178CEA97E00E9437178EEA98E0F5
:109EB0000E9437178CEA97E00E9437178EE298E0ED
:109EC0000E9437178AE390E00E949258EC011A82B0
:109ED0001B821C821D821E821F82188619861A868A
:109EE0001B861C861D861E861F86188A198A1A8A5A
:109EF0001B8A1C8A1D8A1E8A1F8A188E198E1A8E2A
:109F00001B8E1C8E1D8E1E8E1F8E18A219A21AA2C9
:109F10001BA21CA21DA21EA21FA218A619A61AA649
:109F20001BA61CA61DA61EA61FA618AA19AA1AAA19
:109F30001BAA1CAA1DAA1EAA1FAA18AE19AE65E26A
:109F400072E08EEA98E00E94BA598C01DC018C9193
:109F50008654823008F0EEC16EEA77E0C8010E94B4
:109F6000D361892B09F49EC161EB77E0C8010E949F
:109F7000D361892B09F496C165EB77E0C8010E9493
:109F8000D361892B09F491C168EB77E0C8010E9485
:109F9000D361892B09F489C16CEB77E0C8010E9479
:109FA000D361892B09F484C160EC77E0C8010E9479
:109FB000D361892B09F47FC164EC77E0C8010E946A
:109FC000D361892B09F477C167EC77E0C8010E945F
:109FD000D361892B09F472C16BEC77E0C8010E9450
:109FE000D361892B09F46DC16FEC77E0C8010E9441
:109FF000D361892B09F468C163ED77E0C8010E9441
:10A00000D361892B09F463C167ED77E0C8010E9431
:10A01000D361892B09F45EC16BED77E0C8010E9422
:10A02000D361892B09F459C16FED77E0C8010E9413
:10A03000D361892B09F454C163EE77E0C8010E9413
:10A04000D361892B09F44FC167EE77E0C8010E9404
:10A05000D361892B09F44AC16BEE77E0C8010E94F5
:10A06000D361892B09F445C16FEE77E0C8010E94E6
:10A07000D361892B09F440C163EF77E0C8010E94E6
:10A08000D361892B09F43BC167EF77E0C8010E94D7
:10A09000D361892B09F436C16BEF77E0C8010E94C8
:10A0A000D361892B09F431C16FEF77E0C8010E94B9
:10A0B000D361892B09F42CC163E078E0C8010E94C8
:10A0C000D361892B09F427C167E078E0C8010E94B9
:10A0D000D361892B09F422C16BE078E0C8010E94AA
:10A0E000D361892B09F41DC16FE078E0C8010E949B
:10A0F000D361892B09F418C163E178E0C8010E949B
:10A10000D361892B09F013C188EB90E09093010291
:10A11000809300020115110509F412C1F801808134
:10A12000883541F4C80101960E94B7596A837B8340
:10A130008C839D83D8018C91893541F4C8010196A7
:10A140000E94B7596E837F8388879987F801808141
:10A150008A3541F4C80101960E94B7596A877B8706
:10A160008C879D87D8018C91813451F4C801019668
:10A170000E94B7590E9467606E877F87888B998B92
:10A18000F8018081823451F4C80101960E94B759C8
:10A190000E9467606A8B7B8B8C8B9D8BD8018C9126
:10A1A000833451F4C80101960E94B7590E94676038
:10A1B0006E8B7F8B888F998FF8018081833541F476
:10A1C000C80101960E94B7596A8F7B8F8C8F9D8F33
:10A1D000D8018C91803551F4C80101960E94B7597D
:10A1E0000E9467606E8F7F8F88A399A3F80180819A
:10A1F000863551F4C80101960E94B7590E946760E4
:10A200006AA37BA38CA39DA3D8018C91873551F4BD
:10A21000C80101960E94B7590E9467606EA37FA390
:10A2200088A799A7F8018081853451F4C801019667
:10A230000E94B7590E9467606AA77BA78CA79DA759
:10A24000D8018C91843551F4C80101960E94B75908
:10A250000E9467606EA77FA788AB99ABF8018081E9
:10A260008D3451F4C80101960E94B7590E9467606D
:10A270006AAB7BAB8CAB9DABD8018C91813551F433
:10A28000C80101960E94B7590E9467606EAB7FAB10
:10A2900088AF99AF67E178E090E080E00E94BA591A
:10A2A0008C0138CF90E080E031CF81E090E02ECF7C
:10A2B0008CE190E02BCF8DE690E028CF8FE690E008
:10A2C00025CF80E790E022CF81E790E01FCF82E7A3
:10A2D00090E01CCF83E790E019CF84E790E016CFA1
:10A2E00088E790E013CF89E790E010CF8AE790E00D
:10A2F0000DCF83E890E00ACF84E890E007CF8DE8A7
:10A3000090E004CF8EE890E001CF8FE890E0FECEA1
:10A3100080E990E0FBCE81EA90E0F8CE85EB90E01A
:10A32000F5CE86EB90E0F2CE87EB90E0EFCE8FEFAC
:10A330009FEFECCE8FEF9FEF90930102809300028E
:10A340000E942A16FC0114A90E94691E80909B0994
:10A3500090909C09A0909D09B0909E09CEA8DFA87E
:10A36000E8ACF9AC0E942A16DC019296CD92DD92FF
:10A37000ED92FC92959780910002909101028230BB
:10A38000910508F40CC59C012F5631092530310583
:10A3900008F405C5552453948437910509F0512CD0
:10A3A000112309F400C58D36910509F4FCC49C0104
:10A3B000285731092330310508F4F5C4855B91092C
:10A3C000039708F4F0C486E693E00E9437170E94D2
:10A3D0002A160E94C819CE0141D71092780910920E
:10A3E000770980917A098111A4C00E942A16FC0184
:10A3F00084A9882309F49DC00E94DB2DEC01FC0197
:10A40000E45AFC4F108240960E94A111CE018A5559
:10A410009F4F0E94A111CE01845C9E4F0E94A1110A
:10A420000E94B3158C010F5F1F4FC1E0D0E0D8012F
:10A430008D918D018823D9F088E993E00E94371728
:10A4400081E398E00E943717CE010E9432178EE216
:10A4500098E00E94371760E08C2F0E94660970E038
:10A4600060E0CE010E94F019F80131971082F801E6
:10A4700087A98823F9F088E993E00E94371788E4D8
:10A4800098E00E943717CE010E9432178EE298E0C2
:10A490000E94371761E08C2F0E94930960E08C2F97
:10A4A0000E94660961E070E0CE010E94F019D801B7
:10A4B000D7961C922196C533D10509F0B8CF0E94DA
:10A4C000591520913A0E30E0C901880F991F820F6B
:10A4D000931FFC01E755F24F80818F7B8083209191
:10A4E0003D0E30E0C901880F991F820F931FFC01B8
:10A4F000E755F24F80818F7B80832091400E30E0C2
:10A50000C901880F991F820F931FFC01E755F24F75
:10A5100080818F7B80832091430E30E0C901880FBA
:10A52000991F820F931FFC01E755F24F80818F7BAB
:10A5300080830E942A16FC0184A980937A090E94D4
:10A54000691E20917D0930917E09DC0112968D9162
:10A550009C912817390791F10E94691EFC018281A4
:10A56000938190937E0980937D090E94691E2091BA
:10A570007B0930917C09DC0114968D919C91281700
:10A580003907A1F00E94691EFC0184819581909396
:10A590007C0980937B090E94DB2DEC010E949E2A9E
:10A5A000CE010E94732ACE010E94482A0E94DB2D10
:10A5B0000E9401290E94571F0E94271F0E94250AFE
:10A5C00000918309109184092091850930918609B1
:10A5D000601771078207930708F0FDC20E94250AE1
:10A5E0006093830970938409809385099093860909
:10A5F0000E94A7089ECB209781F48EE593E00E94ED
:10A6000037170E942A160E94C8190E942A16DC01D8
:10A6100097967C926E929697DECEE0900002F09034
:10A620000102BFEFEB16FB0671F48EE593E00E948A
:10A6300037170E942A160E94C8190E942A16FC0188
:10A6400077A266A2C8CEE114F10409F083C080911C
:10A65000AC089091AD08892B61F482E090E062D55E
:10A6600028E433E0DC012D933C939093AD08809374
:10A67000AC080091AC081091AD08B1E7EB16F104FD
:10A6800009F09EC08091A2089091A308892B61F4E3
:10A6900082E090E047D526E133E0FC01318320835E
:10A6A0009093A3088093A2080091A2081091A30898
:10A6B000F9E7EF16F10409F09EC080919808909197
:10A6C0009908892B61F482E090E02CD5E4EEF2E069
:10A6D000DC01ED93FC939093990880939808009186
:10A6E000980810919908F0E9EF16F10409F09EC05E
:10A6F00080918E0890918F08892B61F482E090E020
:10A7000011D5E2EBF2E0DC01ED93FC9390938F081E
:10A7100080938E0800918E0810918F08F8EBEF1649
:10A72000F10409F09EC08091840890918508892BDE
:10A7300061F482E090E0F6D4E0E8F2E0DC01ED9331
:10A74000FC9390938508809384080091840810916D
:10A75000850887C0BCE1EB16F104B9F48091AA0822
:10A760009091AB08892B61F482E090E0DBD42EE37A
:10A7700033E0FC01318320839093AB088093AA08D7
:10A780000091AA081091AB0878CFFDE6EF16F1040E
:10A7900009F083C08091A8089091A908892B61F4E1
:10A7A00082E090E0BFD424E333E0DC012D933C93BE
:10A7B0009093A9088093A8080091A8081091A9086F
:10A7C000F2E7EF16F10409F083C08091A0089091A0
:10A7D000A108892B61F482E090E0A4D42CE033E05E
:10A7E000DC012D933C939093A1088093A0080091E5
:10A7F000A0081091A108FAE7EF16F10409F083C050
:10A800008091960890919708892B61F482E090E0FE
:10A8100089D4EAEDF2E0DC01ED93FC939093970884
:10A82000809396080091960810919708F1EAEF1628
:10A83000F10409F083C080918C0890918D08892BD8
:10A8400061F482E090E06ED4E8EAF2E0DC01ED939E
:10A85000FC9390938D0880938C0800918C08109144
:10A860008D080115110509F045C18EE593E00E94A0
:10A8700037170E942A160E94C8190E942A16DC0166
:10A8800097967C926E9296978BE198E00E94BA160A
:10A890008EE298E00E94BA169ECDBFE6EB16F10458
:10A8A00009F068C08091A6089091A708892B61F4EF
:10A8B00082E090E037D42AE233E0FC013183208348
:10A8C0009093A7088093A6080091A6081091A70866
:10A8D000B3E7EB16F10409F0BBC080919E0890919C
:10A8E0009F08892B61F482E090E01CD422E033E0E1
:10A8F000FC013183208390939F0880939E080091F0
:10A900009E0810919F08FDE8EF16F10409F0BBC006
:10A910008091940890919508892B61F482E090E0F1
:10A9200001D4E0EDF2E0DC01ED93FC939093950807
:10A93000809394080091940810919508F5EBEF1618
:10A94000F10409F0BBC080918A0890918B08892B93
:10A9500061F482E090E0E6D3EEE9F2E0DC01ED9311
:10A96000FC9390938B0880938A0800918A08109139
:10A970008B0877CFF0E7EF16F10409F066C08091FD
:10A98000A4089091A508892B61F482E090E0CAD3D5
:10A9900020E233E0DC012D933C939093A508809353
:10A9A000A4080091A4081091A508B8E7EB16F104DB
:10A9B00009F07ECE80919A0890919B08892B51F4E2
:10A9C00082E090E0AFD3FC013182208290939B081B
:10A9D00080939A0800919A0810919B08FFE8EF165F
:10A9E000F10409F080CE8091900890919108892B14
:10A9F00061F482E090E096D3ECEBF2E0DC01ED93C1
:10AA0000FC93909391088093900800919008109186
:10AA10009108F7EBEF16F10409F080CE80918608DB
:10AA200090918708892B61F482E090E07BD3EAE87B
:10AA3000F2E0DC01ED93FC93909387088093860805
:10AA400000918608109187080CCF10E000E015CE29
:10AA5000F4E7EF16F10409F0A8CF80919C089091DB
:10AA60009D08892B61F482E090E05CD328EF32E00E
:10AA7000DC012D933C9390939D0880939C0800915A
:10AA80009C0810919D08FEE8EF16F10409F0A6CF8E
:10AA90008091920890919308892B61F482E090E074
:10AAA00041D3E6ECF2E0DC01ED93FC939093930844
:10AAB000809392080091920810919308F6EBEF169C
:10AAC000F10409F0A6CF8091880890918908892B1C
:10AAD00061F482E090E026D3E4E9F2E0DC01ED935A
:10AAE000FC939093890880938808009188081091BE
:10AAF0008908B7CE8AE593E00E9437170E942A168C
:10AB00000E94C8190E942A16FC0117A216A2F12C55
:10AB1000E12C2FEFE21AF20A31E0E316F10441F0E2
:10AB200086E593E00E9437170E942A160E94C819F2
:10AB3000D801ED91FC910480F581E02DBE01C801A2
:10AB400019950E942A16FC01C6A0D7A00E942A16B9
:10AB5000DC01D4968C9181110AC0E814F9043CF40C
:10AB6000C114D10421F0F2E0CF16D10491F68CE0AB
:10AB70009DE00E940108181619062CF48CE09DE057
:10AB80000E94DF07F4CFCD2809F4F7C0552099F0D3
:10AB90000E94691E8091970990919809A091990946
:10ABA000B0919A090197A105B10529F40E942A16CE
:10ABB00021E0FC0124AB8EE493E00E9437178EE580
:10ABC00098E00E9437170E942A16FC0186A197A1DF
:10ABD0000E943217D6C0AB01BC01401B510B620B67
:10ABE000730B8091020290910302092E000CAA0BB4
:10ABF000BB0B84179507A607B70708F0F9CC0E948E
:10AC00002A16DC01D4968C91882309F481C086E74A
:10AC100093E00E9437170E942A160E94C8190E94CA
:10AC2000DB2DEC01FC01E95CFC4F8081882309F4F9
:10AC300072C00E942A168C01CE018E529E4F0E9435
:10AC4000370DF80166877787808B918BFE01E85C72
:10AC5000FC4F8081882309F46FC00E942A168C0162
:10AC6000CE018E5F9D4F0E94370DF801628B738B72
:10AC7000848B958BFE01E75CFC4F8081882309F46F
:10AC80006CC00E942A168C01CE018E5C9D4F0E94E2
:10AC9000370DF801668B778B808F918F0E942A1673
:10ACA0000E94D11C0E94DB2D0E942B1C0E942A16A0
:10ACB0000E9471160E942A160E940A1B0E94691E99
:10ACC00080918F0990919009A0919109B09192097A
:10ACD0000197A105B10541F08EE693E00E94371778
:10ACE0000E942A160E94C81980917F0990918009BC
:10ACF000A0918109B09182090196A11DB11D809397
:10AD00007F0990938009A0938109B093820966CC52
:10AD100082E793E07ECF0E942A16FE01EE59FF4F94
:10AD20004081518162817381DC011E964D935D9358
:10AD30006D937C9351978ACF0E942A16FE01E850AA
:10AD4000FF4F4081518162817381DC0152964D93A6
:10AD50005D936D937C9355978DCF0E942A16C257B1
:10AD6000DE4F488159816A817B81DC0156964D9383
:10AD70005D936D937C93599791CF82E593E00E9408
:10AD800037170E942A160E94C8190E942A16DC0151
:10AD900092961D921D921D921C9295971CCB552444
:10ADA0005394111110CB0E94691E80918F099091CC
:10ADB0009009A0919109B09192090197A105B1055F
:10ADC00009F419CC552009F416CC82E693E00E94D0
:10ADD00037170E942A160E94C8190E942A162FE0CF
:10ADE00030E0FC0137A326A3F6CA82E89EE00E9469
:10ADF000661D82E79EE00E94661D82E69EE00E943C
:10AE0000661D82E59EE00E94661D82EC9EE00E9427
:10AE1000661D82EB9EE00E94661D82EA9EE00E9413
:10AE2000661D82E99EE00E94661D82E09FE00E940E
:10AE3000661D82EF9EE00E94661D82EE9EE00E94EB
:10AE4000661D82ED9EE00E94661D82E49FE00E94E6
:10AE5000661D82E39FE00E94661D82E29FE00E94E1
:10AE6000661D82E19FE00E94661D82E89FE00E94CD
:10AE7000661D82E79FE00E94661D82E69FE00E94B9
:10AE8000661D82E59FE00E94661D82EC9FE00E94A5
:10AE9000661D82EB9FE00E94661D82EA9FE00E9491
:10AEA000661D82E99FE00E94661D82E090E10E949B
:10AEB000661D82EF9FE00E94661D82EE9FE00E9469
:10AEC000661D82ED9FE00E94661D82E490E10E9473
:10AED000661D82E390E10E94661D82E290E10E947D
:10AEE000661D82E190E10E94661D82E890E10E9469
:10AEF000661D82E790E10E94661D82E690E10E9455
:10AF0000661D82E590E10E94661D82EC90E10E9440
:10AF1000661D82EB90E10E94661D82EA90E10E942C
:10AF2000661D82E990E10E94661D82E091E10E9427
:10AF3000661D82EF90E10E94661D82EE90E10E9404
:10AF4000661D82ED90E10E94661D82E491E10E94FF
:10AF5000661D82E391E10E94661D82E291E10E94FA
:10AF6000661D82E191E10E94661D82E891E10E94E6
:10AF7000661D82E791E10E94661D82E691E10E94D2
:10AF8000661D82E591E10E94661D82EC91E10E94BE
:10AF9000661D82EB91E10E94661D82EA91E10E94AA
:10AFA000661D82E991E10E94661D82E092E10E94A5
:10AFB000661D82EF91E10E94661D82EE91E10E9482
:10AFC000661D82ED91E10E94661D82E492E10E947D
:10AFD000661D82E392E10E94661D82E292E10E9478
:10AFE000661D82E192E10E94661D82E892E10E9464
:10AFF000661D82E792E10E94661D82E692E10E9450
:10B00000661D82E592E10E94661D82EC92E10E943B
:10B01000661D82EB92E10E94661D82EA92E10E9427
:10B02000661D82E992E10E94661D82E093E10E9422
:10B03000661D82EF92E10E94661D82EE92E10E94FF
:10B04000661D82ED92E10E94661D82E493E10E94FA
:10B05000661D82E393E10E94661D82E293E10E94F5
:10B06000661D82E193E10E94661D82E893E10E94E1
:10B07000661D82E793E10E94661D82E693E10E94CD
:10B08000661D82E593E10E94661D82EC93E10E94B9
:10B09000661D82EB93E10E94661D82EA93E10E94A5
:10B0A000661D82E993E10E94661D82E094E10E94A0
:10B0B000661D82EF93E10E94661D82EE93E10E947D
:10B0C000661D82ED93E10E94661D82E494E10E9478
:10B0D000661D82E394E10E94661D82E294E10E9473
:10B0E000661D82E194E10C94661DEF920F931F930D
:10B0F000CF93DF93E80134E047FD34E1042E000CE8
:10B10000550B57FF03C0519541955109E32E022F6E
:10B11000242FAE01ABD1CE01DF91CF911F910F91C2
:10B12000EF9008950F931F93CF93DF938230910593
:10B1300010F482E090E0E0914C14F0914D1430E076
:10B1400020E0B0E0A0E0309799F42115310509F432
:10B150004AC0281B390B24303105D8F58A819B81E0
:10B160006115710589F1FB0193838283FE0111C092
:10B17000408151810281138148175907E0F0481737
:10B18000590799F4109761F012960C931297139641
:10B190001C933296CF01DF91CF911F910F910895AB
:10B1A00000934C1410934D14F4CF2115310551F038
:10B1B0004217530738F0A901DB019A01BD01DF01F5
:10B1C000F801C1CFEF01F9CF90934D1480934C1447
:10B1D000CDCFFE01E20FF31F8193919322503109ED
:10B1E00039832883D7CF20914A1430914B14232BD5
:10B1F00041F4209106023091070230934B142093C2
:10B200004A1420910402309105022115310541F4C0
:10B210002DB73EB74091080250910902241B350B0F
:10B22000E0914A14F0914B14E217F307A0F42E1B9F
:10B230003F0B2817390778F0AC014E5F5F4F24179A
:10B24000350748F04E0F5F1F50934B1440934A143C
:10B25000819391939FCFF0E0E0E09CCFCF93DF9379
:10B260000097E9F0FC01329713821282A0914C14EE
:10B27000B0914D14ED0130E020E01097A1F4208151
:10B280003181820F931F20914A1430914B1428175B
:10B29000390709F061C0F0934B14E0934A14DF9131
:10B2A000CF910895EA01CE17DF07E8F54A815B8167
:10B2B0009E0141155105B1F7E901FB83EA834991EC
:10B2C0005991C40FD51FEC17FD0761F4808191815E
:10B2D0000296840F951FE901998388838281938167
:10B2E0009B838A83F0E0E0E012968D919C91139706
:10B2F0000097B9F52D913C911197CD010296820FDF
:10B30000931F20914A1430914B142817390739F6AE
:10B31000309751F510924D1410924C14B0934B1479
:10B32000A0934A14BCCFD383C28340815181840F40
:10B33000951FC817D90761F44E5F5F4F88819981C7
:10B34000480F591F518340838A819B819383828355
:10B350002115310509F0B0CFF0934D14E0934C1452
:10B360009ECFFD01DC01C0CF13821282D7CF6627AA
:10B370007727F4C148E454E100C0FA01A191B081FB
:10B38000009719F41097E1F0CD01DC01CD010D908B
:10B39000002011F4C00113C0FB012191222319F0F8
:10B3A0002015D9F7F3CFFB012191201519F41E9236
:10B3B000119606C02223C1F70D900020A1F7D001FD
:10B3C000FA01A193B0830895BB274A3031F4992341
:10B3D00022F4BDE2909581959F4F30C0BB272A3063
:10B3E00051F4992342F4BDE2909580957095619552
:10B3F0007F4F8F4F9F4F01C0BB27FA01A62F6217C7
:10B40000710581059105330B30FB66F0AA27660FA5
:10B41000771F881F991FAA1FA21710F0A21B639500
:10B420003850A9F7A05DAA3308F0A95DA19336F7BB
:10B43000B111B1931082CA01DEC3BB27FB015527AE
:10B44000AA27880F991FAA1FA41710F0A41B839581
:10B450005051B9F7A05DAA3308F0A95DA1930097F8
:10B4600079F7B111B1931192CB01C5C38F929F921D
:10B47000AF92BF92CF92DF92EF92FF920F931F9302
:10B48000CF93DF9300D000D000D0CDB7DEB76A01F4
:10B49000F22EB02E102FFBE3AF2EA01608F41BE304
:10B4A0001F5F012F27E0AE014F5F5F4FACD2BC01A1
:10B4B0008981982F9970913009F44EC09BE2E1FC8C
:10B4C00004C09E2D9170E0FC49C05E2D5071E82FA4
:10B4D000E87083FF55C084E0911101C083E0EF2D37
:10B4E000E81B8F1508F0E0E0D6018E2F20E25523EF
:10B4F000C9F1992329F0D6019C93C60101966C01EC
:10B5000096012D5F3F4FE2FE33C08EE4D6018C934F
:10B5100091E411969C93119712968C93D9018E2FDA
:10B5200090E281112AC0E20FF32FF11D10828EEFFD
:10B530009FEF29960FB6F894DEBF0FBECDBFDF9107
:10B54000CF911F910F91FF90EF90DF90CF90BF9020
:10B55000AF909F908F9008959DE2B7CF90E2B5CFC6
:10B560002D9381508111FCCFCE0ED11CE0E0C1CFD4
:10B570008EE6D6018C9391E6CCCF9D938150D1CFAE
:10B58000482F447082FF3DC084E0911101C083E0E8
:10B590008F1510F4EF2DE81BD6018E2F20E25523D6
:10B5A00009F1992329F0D6019C93C60101966C01FB
:10B5B00096012D5F3F4FE2FE1BC089E4D6018C93BC
:10B5C0008EE411968C93119786E412968C93D90190
:10B5D0008E2F90E2882309F4A6CF9D938150FACF55
:10B5E0002D9381508111FCCFCE0ED11CE0E0D9CF3C
:10B5F00089E6D6018C938EE611968C93119786E698
:10B60000E4CF9B0177FF02C030E020E0A1E0B0E092
:10B61000911102C0B0E0A0E0F9013196AE0FBF1F5A
:10B620008B2C912CBB2009F461C05401EFEFAE1AB2
:10B63000BE0AAA0DBB1DFA161B0619F014F04F2DF9
:10B640004A1B511188C0E3FC59C07601A42FB0E217
:10B65000A1114FC0C40ED11C992309F45BC040E076
:10B66000D6011196F60190836D01552309F448C067
:10B67000012F060F9A81582F507184FF03C0913318
:10B6800009F4015010160CF047C0093008F008E02A
:10B69000EEE2FE2E5B01A01AB1088501919481941F
:10B6A00091082F3F320729F4D601FC92F60131961A
:10B6B0006F016217730794F1021713077CF5DB0122
:10B6C000A21BB30BAA24A394B12CAC0EBD1EAA0DD1
:10B6D000BB1D11968C9121503109D6011196281568
:10B6E0003905F4F0F60180836D01DBCFB12CA12C7C
:10B6F000A0CFF701B1937F01A150AACF9111B0CF94
:10B70000D601942F50E302C05D9391509111FCCF6C
:10B71000C40ED11C40E0ACCF01E0BACF80E3DBCF58
:10B720006217730731F4963388F4953311F4552377
:10B7300069F0F6018083FD01842F90E2811108C039
:10B74000A40FB11D1C9290E080E0F3CE81E3F1CF15
:10B7500091938150F3CF911183CF8ACF8F929F9293
:10B76000AF92BF92CF92DF92EF92FF920F931F930F
:10B77000CF93DF935C017B016115710519F0DB014B
:10B780008D939C9385010F5F1F4FF501D0818D2F05
:10B7900090E011D26C01892BA9F5DD32A9F50F5F7C
:10B7A0001F4FD5011196DC91C1E05801F1E0AF1AAD
:10B7B000B10843E050E06CEE70E0C50104D2892B83
:10B7C00061F5680182E0C80ED11C45E050E067EEEB
:10B7D00070E0C601F8D1892B21F4680197E0C90E09
:10B7E000D11CE114F10419F0D701CD92DC9260E094
:10B7F00070E080E89FEFC111F9C060E070E080E880
:10B800009FE7F4C05801BECFDB3229F485010E5FFB
:10B810001F4FF501D181C0E0C8CF43E050E064EE96
:10B8200070E0C501D0D1892BE9F0F80110E000E00B
:10B8300020E030E0A9015F01B0ED8B2E8D0E89E094
:10B840008815C0F19C2E689491F88C2F8870C2FFE7
:10B8500016C0811102C00F5F1F4F3196D501DC91D8
:10B86000C92DE9CFE114F10429F00E5F1F4FF70154
:10B870001183008360E070E080EC9FE7B7C088230D
:10B8800011F001501109A5E0B0E013D39B01AC0108
:10B89000220F331F441F551F280D311D411D511DFF
:10B8A000283999E93907490799E15907B0F2C66083
:10B8B0009C2ED3CFAEEF8A1206C0C3FD3CC09C2E97
:10B8C000689493F8CACFDF7DD534A9F580818D3295
:10B8D00039F4C061DF011296818162E070E006C038
:10B8E000DF018B32C1F3119661E070E080535D019E
:10B8F000A61AB70A8A30F8F4E0E8CE16ECE0DE06C5
:10B900005CF4B601660F771F660F771FC60ED71E51
:10B91000CC0CDD1CC80ED11C5D01FFEFAF1ABF0AB5
:10B920008C9180538A3098F1C4FF03C0D194C194A4
:10B93000D1080C0D1D1DC1FF09C0E114F10431F047
:10B9400081E0A81AB108D701AD92BC92CA01B90131
:10B9500066D1C370C33009F490584B015C0120E0FC
:10B9600030E0A90158D1882309F43EC0CBE1D1E0F1
:10B9700017FF05C0119501951109C3E0D1E06E01D3
:10B98000B8E1CB1AD10880E2E82EF12C0EC0D50127
:10B99000B3CFFE0125913591459154910E191F09A0
:10B9A000C501B4019DD14B015C01D501C4010E1547
:10B9B0001F057CF72497F594E794CC16DD06A9F7CC
:10B9C0008A2F880F8B2F881F8F3F41F020E030E0B7
:10B9D000A901C501B4011FD1811106C082E290E026
:10B9E00090934F1480934E14C501B401DF91CF9111
:10B9F0001F910F91FF90EF90DF90CF90BF90AF908D
:10BA00009F908F900895283008F027E03327DA01BF
:10BA1000990F311D87FD916000966105710539F41C
:10BA200032602E5F3D9330E32A95E1F708959F3F02
:10BA300030F080387105610509F03C5F3C5F3D9353
:10BA4000913008F08068911DDF93CF931F930F937F
:10BA5000FF92EF92192F987F9695E92F96959695DC
:10BA6000E90FFF27E758FE4F99273327EE24FF24DD
:10BA7000A701E70105900894079428F4360FE71E04
:10BA8000F81E491F511D660F771F881F991F0694C6
:10BA9000A1F70590079428F4E70EF81E491F561FDA
:10BAA000C11D770F881F991F661F0694A1F7059087
:10BAB000079428F4F80E491F561FC71FD11D880F81
:10BAC000991F661F771F0694A1F70590079420F42D
:10BAD000490F561FC71FD81F990F661F771F881F52
:10BAE0000694A9F784911095177041F0D695C795E3
:10BAF00057954795F794E7941A95C1F7EFE1F1E070
:10BB000068941590159135916591959105907FE216
:10BB10007395E118F10A430B560BC90BD009C0F716
:10BB2000E10CF11E431F561FC91FD01D7EF4703358
:10BB300011F48A95E6CFE894015030F0080F0AF42A
:10BB40000027021708F4202F2395022F7A3328F0BC
:10BB500079E37D932A95E9F710C07D932A9589F6BC
:10BB6000069497956795379517951794E118F10AFC
:10BB7000430B560BC90BD00998F023957E91739512
:10BB80007A3308F070E37C932013B8F77E917061EC
:10BB90007D9330F0839571E37D9370E32A95E1F70F
:10BBA0001124EF90FF900F911F91CF91DF91992772
:10BBB00087FD909508959111F6C0803219F0895053
:10BBC0008550D0F70895FB01DC014150504088F0CA
:10BBD0008D9181341CF08B350CF4805E659161345D
:10BBE0001CF06B350CF4605E861B611171F3990BD0
:10BBF0000895881BFCCFDC01FC01672F719177232E
:10BC0000E1F7329704C07C916D9370836291AE1717
:10BC1000BF07C8F3089540D008F481E00895E89480
:10BC200009C097FB3EF490958095709561957F4F84
:10BC30008F4F9F4F9923A9F0F92F96E9BB27939532
:10BC4000F695879577956795B795F111F8CFFAF442
:10BC5000BB0F11F460FF1BC06F5F7F4F8F4F9F4F73
:10BC600016C0882311F096E911C0772321F09EE8D1
:10BC7000872F762F05C0662371F096E8862F70E037
:10BC800060E02AF09A95660F771F881FDAF7880F11
:10BC90009695879597F90895990F0008550FAA0B67
:10BCA000E0E8FEEF16161706E807F907C0F01216CF
:10BCB0001306E407F50798F0621B730B840B950BD2
:10BCC00039F40A2661F0232B242B252B21F4089527
:10BCD0000A2609F4A140A6958FEF811D811D0895C4
:10BCE0000BD07BC06CD028F071D018F0952309F0F0
:10BCF0005DC062C01124A5C081D0A0F3959FD1F38F
:10BD0000950F50E0551F629FF001729FBB27F00D09
:10BD1000B11D639FAA27F00DB11DAA1F649F66275E
:10BD2000B00DA11D661F829F2227B00DA11D621FAD
:10BD3000739FB00DA11D621F839FA00D611D221F67
:10BD4000749F3327A00D611D231F849F600D211D4B
:10BD5000822F762F6A2F11249F5750408AF0E1F0EE
:10BD600088234AF0EE0FFF1FBB1F661F771F881F37
:10BD700091505040A9F79E3F510570F017C061C027
:10BD80005F3FECF3983EDCF3869577956795B79522
:10BD9000F795E7959F5FC1F7FE2B880F911D96954C
:10BDA000879597F9089599278827089597F99F67A8
:10BDB00080E870E060E008959FEF80EC0895002433
:10BDC0000A941616170618060906089500240A9400
:10BDD00012161306140605060895092E0394000C86
:10BDE00011F4882352F0BB0F40F4BF2B11F460FF15
:10BDF00004C06F5F7F4F8F4F9F4F089557FD90583E
:10BE0000440F551F59F05F3F71F04795880F97FB1E
:10BE1000991F61F09F3F79F08795089512161306D8
:10BE20001406551FF2CF4695F1DF08C01616170607
:10BE30001806991FF1CF869571056105089408953C
:10BE4000E894BB2766277727CB0197F90895F999DE
:10BE5000FECF92BD81BDF89A992780B50895262F0F
:10BE6000F999FECF1FBA92BD81BD20BD0FB6F894DF
:10BE7000FA9AF99A0FBE01960895052E97FB16F4CB
:10BE800000940FD057FD05D024D007FC02D046F413
:10BE900008C050954095309521953F4F4F4F5F4FCB
:10BEA000089590958095709561957F4F8F4F9F4F26
:10BEB000089531D0A59F900DB49F900DA49F800D43
:10BEC000911D11240895B7FFF4CFF3DF821B930B6C
:10BED0000895A1E21A2EAA1BBB1BFD010DC0AA1FCB
:10BEE000BB1FEE1FFF1FA217B307E407F50720F0E3
:10BEF000A21BB30BE40BF50B661F771F881F991F5E
:10BF00001A9469F760957095809590959B01AC01A6
:10BF1000BD01CF010895A29FB001B39FC001A39FAF
:10BF2000700D811D1124911DB29F700D811D112472
:10BF3000911D08955058BB27AA270ED04ECF3FDF42
:10BF400030F044DF20F031F49F3F11F41EF434CF81
:10BF50000EF4E095E7FB2ACFE92F50DF80F3BA1704
:10BF6000620773078407950718F071F49EF568CF90
:10BF70000EF4E0950B2EBA2FA02D0B01B901900104
:10BF80000C01CA01A0011124FF27591B99F0593F48
:10BF900050F4503E68F11A16F040A22F232F342F90
:10BFA0004427585FF3CF469537952795A795F040DE
:10BFB0005395C9F77EF41F16BA0B620B730B840BF3
:10BFC000BAF09150A1F0FF0FBB1F661F771F881FAB
:10BFD000C2F70EC0BA0F621F731F841F48F4879503
:10BFE00077956795B795F7959E3F08F0B3CF9395F2
:10BFF000880F08F09927EE0F9795879508950CD034
:10C00000ECCEE4DE40F0DBDE30F021F45F3F19F0EF
:10C01000CDCE511116CFD0CEF1DE98F39923C9F3CE
:10C020005523B1F3951B550BBB27AA27621773073E
:10C03000840738F09F5F5F4F220F331F441FAA1FF2
:10C04000A9F333D00E2E3AF0E0E830D091505040B2
:10C05000E695001CCAF729D0FE2F27D0660F771F60
:10C06000881FBB1F261737074807AB07B0E809F042
:10C07000BB0B802DBF01FF2793585F4F2AF09E3FD7
:10C08000510568F093CEDDCE5F3FECF3983EDCF3D4
:10C09000869577956795B795F7959F5FC9F7880F50
:10C0A000911D9695879597F90895E1E0660F771FA2
:10C0B000881FBB1F621773078407BA0720F0621B33
:10C0C000730B840BBA0BEE1F88F7E095089504D02C
:10C0D0006894B111B6CE089599DE88F09F5790F01C
:10C0E000B92F9927B751A0F0D1F0660F771F881F9D
:10C0F000991F1AF0BA95C9F712C0B13081F0A0DECD
:10C10000B1E008959DCE672F782F8827B85F39F06A
:10C11000B93FCCF3869577956795B395D9F73EF4FB
:10C1200090958095709561957F4F8F4F9F4F0895A3
:10C13000B3DD08F48FEF0895AFDD880B990B0895F8
:10C14000DB018F939F93B5DEBF91AF91A29F800DCE
:10C15000911DA39F900DB29F900D11240895991BDE
:10C1600079E004C0991F961708F0961B881F7A95EE
:10C17000C9F78095089597FB072E16F4009406D012
:10C1800077FD08D013D007FC05D03EF4909581953B
:10C190009F4F0895709561957F4F0895EE0FFF1F93
:10C1A000881F8BBF0790F691E02D1994AA1BBB1B2B
:10C1B00051E107C0AA1FBB1FA617B70710F0A61BA7
:10C1C000B70B881F991F5A95A9F780959095BC01C8
:10C1D000CD0108954F925F926F927F928F929F92BE
:10C1E000AF92BF92CF92DF92EF92FF920F931F9385
:10C1F000CF93DF938C01009799F4CB01DF91CF911E
:10C200001F910F91FF90EF90DF90CF90BF90AF9074
:10C210009F908F907F906F905F904F900C9492586A
:10C22000FC01E60FF71F9C0122503109E217F307CA
:10C2300008F4ADC0D901CD91DC911197C617D7078D
:10C2400020F1C530D10578F0CE0104978617970705
:10C2500050F0C61BD70B2297C193D1936D937C935B
:10C26000CF010E942E59C801DF91CF911F910F91EC
:10C27000FF90EF90DF90CF90BF90AF909F908F9006
:10C280007F906F905F904F9008955B01AC1ABD0A4C
:10C290004C018C0E9D1EA0914C14B0914D14512C4C
:10C2A000412CF12CE12C109731F580914A1490919A
:10C2B0004B148815990509F05CC04616570608F01E
:10C2C00058C08091040290910502009741F48DB707
:10C2D0009EB74091080250910902841B950BE81704
:10C2E000F90708F054C0F0934B14E0934A14F90195
:10C2F00071836083B8CF8D919C91119712966C9049
:10C30000129713967C901397A815B90559F56C01EF
:10C3100042E0C40ED11CCA14DB0420F1AC014A195E
:10C320005B09DA011296159780F06282738251835D
:10C330004083D9016D937C93E114F10471F0D7012E
:10C340001396FC93EE9312978ECF22968C0F9D1F1F
:10C35000F90191838083F301EFCFF0934D14E093C3
:10C360004C1481CF4816590608F42C017D01D301E5
:10C370009ACFCB010E9492587C01009741F0AE0108
:10C38000B80108D0C8010E942E5987016CCF10E077
:10C3900000E069CFFB01DC0102C001900D92415029
:10C3A0005040D8F70895FB01DC018D910190801970
:10C3B0000110D9F3990B0895FB01DC0101900D9256
:10C3C0000020E1F7089511E0CEE9D1E000E005C0DA
:10C3D000802FFE01E3DE2196011DCF39D10780E0D9
:08C3E0000807B1F7F894FFCF44
:10C3E800FFFF88130000501480002E482E67656EEA
:10C3F800657369734B3135000001000000010000CE
:10C408000001000000200A0D0000362E352E3232C1
:10C41800000052303500523835005238340052315D
:10C42800330052313200523131005231370052312B
:10C438003600523135005230340052383700523706
:10C44800330052373200523731000D0A00200052B3
:10C458003939000D0A002000523939000000000067
:10C468004615781D1E2E0000000047157A1DF91A82
:10C478000000000048157C1D611D000000004915E2
:10C488007E1D341B000000004A15801D6C1500003D
:10C4980000004B15821DD015000000004C15841DAE
:10C4A8000C16000000004D15861D991A00000000AA
:10C4B8004E15881D1916000000004F158A1DC82A40
:10C4C8000000000050158C1D342B00000000511591
:10C4D8006E1D422B0000000052158E1D35410000D4
:10C4E80000005315901D6E41000000005415921D68
:10C4F800A741000000005515941DE0410000000010
:10C508005615961DD043000000005715981D9445F8
:10C518000000000058159A1DB416000000004415CC
:10C52800741D5140000000004515761DF940523039
:10C53800330052303200523037005230310052301E
:10C5480039005238380052383700523038005238E3
:10C558003800523030005238370052303600000070
:10C5680000003808A307D00788080108DF07F30789
:10C57800000000004015701D5239390020737461A5
:10C58800200020637572200020656E6420002068FA
:10C59800616C662000206C656E2000206D696E203D
:10C5A80000206D6178200020737064200020510005
:10C5B800523431005000523231005239392045721C
:10C5C800726F723A20696E76616C6964207061726C
:10C5D800616D657465722069640D0A0052383320F4
:10C5E800002D3839666264313739005238310020FD
:10C5F800584100205842002059410020594200204B
:10C608005A4100205A4200686F6D650D0A006E613C
:10C618006E00696E66006F766600523832005232DC
:10C6280030005239392057696C6C207A65726F2056
:10C6380058005239392057696C6C207A65726F201E
:10C6480059005239392057696C6C207A65726F200D
:10C658005A007469636B2064656C6179004D4F56AC
:10C66800454D454E545F494E544552525550545FBE
:10C678005350454544007370656564486F6D655B4C
:10C68800617869735D005239392043616C6962725F
:10C698006174696F6E206572726F723A20656E649C
:10C6A8002073746F702061637469766520626566B3
:10C6B8006F72652073746172740D0A002061786965
:10C6C800732000206D6F766520746F20737461721B
:10C6D8007420666F722063616C6962726174696F3D
:10C6E8006E005239392074696D656F757420582051
:10C6F800617869730D0A005239392074696D656F64
:10C708007574205920617869730D0A0052393920EF
:10C7180074696D656F7574205A20617869730D0AA4
:10C728000052393920656D657267656E63792073CB
:10C73800746F700D0A00523939206D6F76656D651A
:10C748006E7420646F6E650D0A0020617420737426
:10C75800617274696E6720706F696E74005232334B
:10C76800002063616C6962726174696E67206C6530
:10C778006E67746800207374657020636F756E74DB
:10C788003A200020617420656E6420706F696E74B1
:10C79800002064656163746976617465206D6F74E7
:10C7A8006F7220582064756520746F20006D69735E
:10C7B80073656420737465707300206465616374C5
:10C7C8006976617465206D6F746F72205920647585
:10C7D8006520746F200020646561637469766174F4
:10C7E80065206D6F746F72205A2064756520746FB0
:10C7F8002000523939206572726F720D0A00523961
:10C80800392073746F707065640D0A0052393920CD
:10C818006572726F72200052393920686F6D696EC7
:10C828006720646973706C61636564002058200038
:10C83800202F200020592000205A2000204D2000C1
:10C8480053657269616C20636F6E6E656374696F9E
:10C858006E20737461727465640053657420696E28
:10C868007075742F6F7574707574206661726D625F
:10C878006F74206578707265737300526561642007
:10C88800706172616D6574657273004C6F616420CC
:10C89800544D43206472697665727300496E6974F9
:10C8A80020544D4332313330206472697665727397
:10C8B800004C6F616420544D433231333020706135
:10C8C80072616D6574657273004C6F6164206D6F81
:10C8D80076656D656E742073657474696E67730030
:10C8E800536574206D6F746F7220656E61626C653C
:10C8F80073206F66660053746172742070696E20CD
:10C90800677561726400537461727420696E74652E
:10C91800727275707400436865636B20686F6D6927
:10C928006E67206F6E20626F6F740052393920482D
:10C938004F4D45205A204F4E205354415254555084
:10C948000D0A0052393920484F4D452059204F4E85
:10C9580020535441525455500D0A00523939204839
:10C968004F4D452058204F4E205354415254555056
:10C978000D0A0041524455494E4F205354415254D8
:10C98800555020434F4D504C455445002A004730E0
:10C998000047303000473100473031004732380017
:10C9A80046303900463900463131004631320046BA
:10C9B80031330046313400463135004631360046C1
:10C9C80032300046323100463232004633310046BA
:10C9D80033320046343100463432004634330046A0
:10C9E8003434004636310046383100463832004685
:10C9F80038330046383400200A0D0052393920688F
:10CA0800616E646C6572203D3D204E554C4C0D0A9C
:10CA18000020726573657474696E6720646967695C
:10CA280074616C2070696E00207265736574746936
:10CA38006E6720616E616C6F672070696E002056AA
:02CA48000000EC
:00000001FF
